:020000040800F2
:1000000000500020495F00087187000873870008CE
:1000100075870008778700087987000800000000CE
:100020000000000000000000000000007B870008C6
:100030007D870008000000007F870008995F0008A6
:10004000995F0008995F0008995F0008995F0008B0
:10005000995F0008995F0008995F0008995F0008A0
:10006000995F0008995F0008995F0008995F000890
:10007000995F0008995F0008995F0008995F000880
:10008000995F0008995F0008995F0008995F000870
:1000900081870008995F0008995F0008D96E000801
:1000A000995F0008995F0008995F0008995F000850
:1000B0008D6000081D630008995F0008995F0008C3
:1000C000995F0008995F0008995F0008995F000830
:1000D000995F0008A1540008995F0008995F000823
:1000E0008D2A0008995F0008995F00080000000051
:1000F0000000000000000000000000000000000000
:0C01000000000000000000005FF808F1A3
:1001100010B5054C237833B9044B13B10448AFF341
:1001200000800123237010BDF801002000000000B2
:10013000D0A2000808B5034B1BB103490348AFF335
:10014000008008BD00000000FC010020D0A20008D3
:1001500081F0004102E000BF83F0004330B54FEA78
:1001600041044FEA430594EA050F08BF90EA020FE5
:100170001FBF54EA000C55EA020C7FEA645C7FEA78
:10018000655C00F0E2804FEA5454D4EB5555B8BF9B
:100190006D420CDD2C4480EA020281EA030382EA0C
:1001A000000083EA010180EA020281EA0303362D9E
:1001B00088BF30BD11F0004F4FEA01314FF4801C71
:1001C0004CEA113102D0404261EB410113F0004F83
:1001D0004FEA03334CEA133302D0524263EB43033A
:1001E00094EA050F00F0A780A4F10104D5F1200ED8
:1001F0000DDB02FA0EFC22FA05F2801841F1000133
:1002000003FA0EF2801843FA05F359410EE0A5F106
:1002100020050EF1200E012A03FA0EFC28BF4CF037
:10022000020C43FA05F3C01851EBE37101F00045ED
:1002300007D54FF0000EDCF1000C7EEB00006EEBFA
:100240000101B1F5801F1BD3B1F5001F0CD3490884
:100250005FEA30004FEA3C0C04F101044FEA4452DB
:1002600012F5800F80F09A80BCF1004F08BF5FEA62
:10027000500C50F1000041EB045141EA050130BD42
:100280005FEA4C0C404141EB010111F4801FA4F1E5
:100290000104E9D191F0000F04BF01460020B1FA3A
:1002A00081F308BF2033A3F10B03B3F120020CDA72
:1002B0000C3208DD02F1140CC2F10C0201FA0CF050
:1002C00021FA02F10CE002F11402D8BFC2F1200CB5
:1002D00001FA02F120FA0CFCDCBF41EA0C0190406B
:1002E000E41AA2BF01EB0451294330BD6FEA0404B4
:1002F0001F3C1CDA0C340EDC04F11404C4F120029F
:1003000020FA04F001FA02F340EA030021FA04F3B0
:1003100045EA030130BDC4F10C04C4F1200220FA07
:1003200002F001FA04F340EA0300294630BD21FA45
:1003300004F0294630BD94F0000F83F4801306BF0B
:1003400081F480110134013D4EE77FEA645C18BFFF
:100350007FEA655C29D094EA050F08BF90EA020F96
:1003600005D054EA000C04BF1946104630BD91EA8E
:10037000030F1EBF0021002030BD5FEA545C05D191
:100380004000494128BF41F0004130BD14F58004D0
:100390003CBF01F5801130BD01F0004545F0FE4144
:1003A00041F470014FF0000030BD7FEA645C1ABF79
:1003B000194610467FEA655C1CBF0B46024650EAB0
:1003C000013406BF52EA033591EA030F41F40021DC
:1003D00030BD00BF90F0000F04BF0021704730B562
:1003E0004FF4806404F132044FF000054FF0000137
:1003F00050E700BF90F0000F04BF0021704730B5F8
:100400004FF4806404F1320410F0004548BF4042CC
:100410004FF000013EE700BF42004FEAE2014FEA21
:1004200031014FEA02701FBF12F07F4393F07F4FFC
:1004300081F06051704792F0000F14BF93F07F4F2E
:10044000704730B54FF4607401F0004521F0004171
:1004500020E700BF50EA010208BF704730B54FF0F7
:1004600000050AE050EA010208BF704730B511F0FC
:10047000004502D5404261EB41014FF4806404F134
:1004800032045FEA915C3FF4DCAE4FF003025FEAB6
:10049000DC0C18BF03325FEADC0C18BF033202EB3E
:1004A000DC02C2F1200300FA03FC20FA02F001FA98
:1004B00003FE40EA0E0021FA02F11444C1E600BF37
:1004C00070B54FF0FF0C4CF4E06C1CEA11541DBFEA
:1004D0001CEA135594EA0C0F95EA0C0F00F0DEF8B5
:1004E0002C4481EA030621EA4C5123EA4C5350EA9A
:1004F000013518BF52EA033541F4801143F48013EB
:1005000038D0A0FB02CE4FF00005E1FB02E506F07B
:100510000042E0FB03E54FF00006E1FB03569CF0D0
:10052000000F18BF4EF0010EA4F1FF04B6F5007FD6
:1005300064F5407404D25FEA4E0E6D4146EB060648
:1005400042EAC62141EA55514FEAC52040EA5E50D1
:100550004FEACE2EB4F1FD0C88BFBCF5E06F1ED87B
:10056000BEF1004F08BF5FEA500E50F1000041EBB2
:10057000045170BD06F0004646EA010140EA02005F
:1005800081EA0301B4EB5C04C2BFD4EB0C0541EA81
:10059000045170BD41F480114FF0000E013C00F396
:1005A000AB8014F1360FDEBF002001F0004170BDBA
:1005B000C4F10004203C35DA0C341BDC04F11404D3
:1005C000C4F1200500FA05F320FA04F001FA05F25F
:1005D00040EA020001F0004221F0004110EBD3702C
:1005E00021FA04F642EB06015EEA430E08BF20EA58
:1005F000D37070BDC4F10C04C4F1200500FA04F3FB
:1006000020FA05F001FA04F240EA020001F000418C
:1006100010EBD37041F100015EEA430E08BF20EAFF
:10062000D37070BDC4F1200500FA05F24EEA020E47
:1006300020FA04F301FA05F243EA020321FA04F076
:1006400001F0004121FA04F220EA020000EBD3702D
:100650005EEA430E08BF20EAD37070BD94F0000F2D
:100660000FD101F00046400041EB010111F4801F61
:1006700008BF013CF7D041EA060195F0000F18BF12
:10068000704703F00046520043EB030313F4801F4E
:1006900008BF013DF7D043EA0603704794EA0C0F08
:1006A0000CEA135518BF95EA0C0F0CD050EA41061E
:1006B00018BF52EA4306D1D181EA030101F000419B
:1006C0004FF0000070BD50EA410606BF10461946C3
:1006D00052EA430619D094EA0C0F02D150EA0136CF
:1006E00013D195EA0C0F05D152EA03361CBF104610
:1006F00019460AD181EA030101F0004141F0FE41AF
:1007000041F470014FF0000070BD41F0FE4141F432
:10071000780170BD70B54FF0FF0C4CF4E06C1CEA32
:1007200011541DBF1CEA135594EA0C0F95EA0C0FE7
:1007300000F0A7F8A4EB050481EA030E52EA0335A2
:100740004FEA013100F088804FEA03334FF08055C3
:1007500045EA131343EA12634FEA022245EA1115F0
:1007600045EA10654FEA00260EF000419D4208BFA1
:10077000964244F1FD0404F5407402D25B084FEA4E
:100780003202B61A65EB03055B084FEA32024FF4FA
:1007900080104FF4002CB6EB020E75EB030E22BF57
:1007A000B61A754640EA0C005B084FEA3202B6EB17
:1007B000020E75EB030E22BFB61A754640EA5C00C6
:1007C0005B084FEA3202B6EB020E75EB030E22BF56
:1007D000B61A754640EA9C005B084FEA3202B6EB57
:1007E000020E75EB030E22BFB61A754640EADC0016
:1007F00055EA060E18D04FEA051545EA16754FEA78
:1008000006164FEAC30343EA52734FEAC2025FEA95
:100810001C1CC0D111F4801F0BD141EA00014FF024
:1008200000004FF0004CB6E711F4801F04BF0143F5
:100830000020B4F1FD0C88BFBCF5E06F3FF6AFAE11
:10084000B5EB030C04BFB6EB020C5FEA500C50F1A1
:10085000000041EB045170BD0EF0004E4EEA113124
:1008600014EB5C04C2BFD4EB0C0541EA045170BD2B
:1008700041F480114FF0000E013C90E645EA060E6F
:100880008DE60CEA135594EA0C0F08BF95EA0C0F9D
:100890003FF43BAF94EA0C0F0AD150EA01347FF4E5
:1008A00034AF95EA0C0F7FF425AF104619462CE7BC
:1008B00095EA0C0F06D152EA03353FF4FDAE10461F
:1008C000194622E750EA410618BF52EA43067FF470
:1008D000C5AE50EA41047FF40DAF52EA43057FF400
:1008E000EBAE12E74FF0FF3C06E000BF4FF0010C0B
:1008F00002E000BF4FF0010C4DF804CD4FEA410C6F
:100900007FEA6C5C4FEA430C18BF7FEA6C5C1BD03B
:1009100001B050EA410C0CBF52EA430C91EA030FBC
:1009200002BF90EA020F0020704710F1000F91EA19
:10093000030F58BF994208BF90422CBFD8176FEAE7
:10094000E37040F0010070474FEA410C7FEA6C5CB5
:1009500002D150EA013C07D14FEA430C7FEA6C5CBC
:10096000D6D152EA033CD3D05DF8040B704700BFE8
:100970008446104662468C461946634600E000BF36
:1009800001B5FFF7B7FF002848BF10F1000F01BD08
:100990004DF808EDFFF7F4FF0CBF012000205DF8D3
:1009A00008FB00BF4DF808EDFFF7EAFF34BF012058
:1009B00000205DF808FB00BF4DF808EDFFF7E0FFF1
:1009C00094BF012000205DF808FB00BF4DF808ED42
:1009D000FFF7CEFF94BF012000205DF808FB00BFA9
:1009E0004DF808EDFFF7C4FF34BF012000205DF88B
:1009F00008FB00BF4FEA410C7FEA6C5C02D150EA71
:100A0000013C0AD14FEA430C7FEA6C5C02D152EA06
:100A1000033C02D14FF0000070474FF001007047D7
:100A20004FEA410212F5001215D211D56FF4787316
:100A3000B3EB625212D94FEAC12343F0004343EAB9
:100A4000505311F0004F23FA02F018BF4042704794
:100A50004FF00000704750EA013005D111F000401E
:100A600008BF6FF0004070474FF00000704700BFB4
:100A70004FEA4102B2F1E04324BFB3F5001CDCF1C0
:100A8000FE5C0DD901F0004C4FEAC0024CEA5070F8
:100A9000B2F1004F40EB830008BF20F00100704727
:100AA00011F0804F21D113F13872BCBF01F000402A
:100AB000704741F480114FEA5252C2F11802C2F15C
:100AC000200C10FA0CF320FA02F018BF40F00100DD
:100AD0004FEAC1234FEAD32303FA0CFC40EA0C008F
:100AE00023FA02F34FEA4303CCE77FEA625307D1CC
:100AF00050EA01331EBF4FF0FE4040F44000704703
:100B000001F0004040F0FE4040F40000704700BF9C
:100B100080F0004002E000BF81F0004142001FBFB2
:100B20005FEA410392EA030F7FEA226C7FEA236CBB
:100B30006AD04FEA1262D2EB1363C1BFD2184140B0
:100B400048404140B8BF5B42192B88BF704710F046
:100B5000004F40F4000020F07F4018BF404211F0E9
:100B6000004F41F4000121F07F4118BF494292EA51
:100B7000030F3FD0A2F1010241FA03FC10EB0C007D
:100B8000C3F1200301FA03F100F0004302D549420A
:100B900060EB4000B0F5000F13D3B0F1807F06D3B7
:100BA00040084FEA310102F10102FE2A51D2B1F1AF
:100BB000004F40EBC25008BF20F0010040EA0300A4
:100BC0007047490040EB000010F4000FA2F1010251
:100BD000EDD1B0FA80FCACF1080CB2EB0C0200FADB
:100BE0000CF0AABF00EBC25052421843BCBFD04029
:100BF0001843704792F0000F81F4000106BF80F4A3
:100C000000000132013BB5E74FEA41037FEA226C65
:100C100018BF7FEA236C21D092EA030F04D092F030
:100C2000000F08BF0846704790EA010F1CBF002064
:100C3000704712F07F4F04D1400028BF40F00040C1
:100C4000704712F100723CBF00F50000704700F0E1
:100C5000004343F0FE4040F4000070477FEA226208
:100C600016BF08467FEA23630146420206BF5FEAD9
:100C7000412390EA010F40F4800070474FF00003D9
:100C800004E000BF10F0004348BF40425FEA000CA0
:100C900008BF704743F0964301464FF000001CE048
:100CA00050EA010208BF70474FF000030AE000BF9E
:100CB00050EA010208BF704711F0004302D54042DC
:100CC00061EB41015FEA010C02BF8446014600204E
:100CD00043F0B64308BFA3F18053A3F50003BCFA69
:100CE0008CF2083AA3EBC25310DB01FA02FC634416
:100CF00000FA02FCC2F12002BCF1004F20FA02F21D
:100D000043EB020008BF20F00100704702F120020F
:100D100001FA02FCC2F1200250EA4C0021FA02F270
:100D200043EB020008BF20EADC7070474FF0FF0C75
:100D30001CEAD0521EBF1CEAD15392EA0C0F93EA70
:100D40000C0F6FD01A4480EA010C400218BF5FEA12
:100D500041211ED04FF0006343EA501043EA511185
:100D6000A0FB01310CF00040B1F5000F3EBF49007F
:100D700041EAD3715B0040EA010062F17F02FD2A83
:100D80001DD8B3F1004F40EBC25008BF20F0010066
:100D9000704790F0000F0CF0004C08BF49024CEA7D
:100DA000502040EA51207F3AC2BFD2F1FF0340EA0F
:100DB000C250704740F400004FF00003013A5DDC80
:100DC00012F1190FDCBF00F000407047C2F10002C1
:100DD000410021FA02F1C2F1200200FA02FC5FEAAE
:100DE000310040F1000053EA4C0308BF20EADC70F8
:100DF000704792F0000F00F0004C02BF400010F46A
:100E0000000F013AF9D040EA0C0093F0000F01F016
:100E1000004C02BF490011F4000F013BF9D041EA38
:100E20000C018FE70CEAD15392EA0C0F18BF93EA3A
:100E30000C0F0AD030F0004C18BF31F0004CD8D164
:100E400080EA010000F00040704790F0000F17BFEB
:100E500090F0004F084691F0000F91F0004F14D031
:100E600092EA0C0F01D142020FD193EA0C0F03D189
:100E70004B0218BF084608D180EA010000F000408C
:100E800040F0FE4040F40000704740F0FE4040F467
:100E9000400070474FF0FF0C1CEAD0521EBF1CEA06
:100EA000D15392EA0C0F93EA0C0F69D0A2EB030224
:100EB00080EA010C49024FEA402037D04FF08053BE
:100EC00043EA111143EA10130CF000408B4238BF83
:100ED0005B0042F17D024FF4000C8B4224BF5B1A91
:100EE00040EA0C00B3EB510F24BFA3EB510340EADF
:100EF0005C00B3EB910F24BFA3EB910340EA9C008D
:100F0000B3EBD10F24BFA3EBD10340EADC001B01FC
:100F100018BF5FEA1C1CE0D1FD2A3FF650AF8B42A0
:100F200040EBC25008BF20F0010070470CF0004CAD
:100F30004CEA50207F32C2BFD2F1FF0340EAC250D8
:100F4000704740F400004FF00003013A37E792F099
:100F5000000F00F0004C02BF400010F4000F013AF7
:100F6000F9D040EA0C0093F0000F01F0004C02BFF2
:100F7000490011F4000F013BF9D041EA0C0195E75B
:100F80000CEAD15392EA0C0F08D142027FF47DAFF4
:100F900093EA0C0F7FF470AF084676E793EA0C0FE4
:100FA00004D14B023FF44CAF08466EE730F0004CE2
:100FB00018BF31F0004CCAD130F000427FF45CAF72
:100FC00031F000437FF43CAF5FE700BF4FF0FF3CE0
:100FD00006E000BF4FF0010C02E000BF4FF0010C33
:100FE0004DF804CD4FEA40024FEA41037FEA226CFC
:100FF00018BF7FEA236C11D001B052EA530C18BF1E
:1010000090EA010F58BFB2EB030088BFC81738BF82
:101010006FEAE17018BF40F0010070477FEA226C70
:1010200002D15FEA402C05D17FEA236CE4D15FEA6C
:10103000412CE1D05DF8040B704700BF84460846A0
:101040006146FFE70FB5FFF7C9FF002848BF10F161
:10105000000F0FBD4DF808EDFFF7F4FF0CBF0120A6
:1010600000205DF808FB00BF4DF808EDFFF7EAFF30
:1010700034BF012000205DF808FB00BF4DF808EDEB
:10108000FFF7E0FF94BF012000205DF808FB00BFE0
:101090004DF808EDFFF7D2FF94BF012000205DF866
:1010A00008FB00BF4DF808EDFFF7C8FF34BF012073
:1010B00000205DF808FB00BF4FEA40024FEA410301
:1010C0007FEA226C02D15FEA402C08D17FEA236CD0
:1010D00002D15FEA412C02D14FF0000070474FF07F
:1010E000010070474FEA4002B2F1FE4F0FD34FF0BC
:1010F0009E03B3EB12620DD94FEA002343F0004385
:1011000010F0004F23FA02F018BF404270474FF032
:101110000000704712F1610F01D1420205D110F0B9
:10112000004008BF6FF0004070474FF0000070476C
:1011300042000ED2B2F1FE4F0BD34FF09E03B3EB41
:10114000126209D44FEA002343F0004323FA02F06D
:1011500070474FF00000704712F1610F01D1420259
:1011600002D14FF0FF3070474FF00000704700BFD2
:1011700040F0BF60024B40F40030D860704700BFC1
:1011800000ED00E010B5C2780378E2B1124AD168F0
:101190004278C943C1F30221C1F10404A2400F24E3
:1011A000807824FA01F101400A430C491201C81861
:1011B000D2B280F8002303F01F005A0901238340B4
:1011C00041F8223010BD01215A0903F01F0301FA32
:1011D00003F320320149F3E700ED00E000E100E015
:1011E000827930B50168037942B3CC43184A03F1E0
:1011F0008043156803F582332540156055682C40FF
:1012000054601C682143196003689468D9430C40FA
:101210009460D4682140D1604179102906D1916849
:1012200019439160D1680B43D36030BD01F1804216
:1012300002F5823211680B43136030BD03F1804325
:1012400003F582331A6822EA0101196030BD00BF3C
:1012500000040140054B1A685B69034004D0024258
:1012600014BF012000207047184670470004014059
:10127000014B5861704700BF00040140034B044A12
:101280005A6002F188325A60704700BF0020024065
:1012900023016745FFF7F2BF084BDA68D10709D48D
:1012A000DA68520708D4DB6813F0100F14BF03206C
:1012B0000420704701207047022070470020024040
:1012C00010B50446FFF7E8FF012806D10CB9052048
:1012D00010BDFFF7E1FF013CF6E7002C08BF052039
:1012E00010BD000070B505464FF400500E46FFF7E4
:1012F000E7FF04280FD1084C4FF40050236943F056
:10130000010323612E80FFF7DBFF236923F0010334
:10131000DB04DB0C236170BD0020024038B50546BC
:101320004FF43020FFF7CCFF042813D10A4C4FF4C0
:101330003020236943F0020323616561236943F090
:1013400040032361FFF7BCFF236923F00203DB04A2
:10135000DB0C236138BD00BF00200240CB782DE9B3
:10136000F041DA0648BF8A780E8803F00F0548BFBF
:10137000154316F0FF0F1AD000214FF0010E4FF069
:101380000F0C02680EFA01F737EA06040BD18C0045
:101390000CFA04F822EA080205FA04F4282B42EABF
:1013A000040225D1476101310829EBD10260FF2EEB
:1013B0001CD900214FF0010E4FF00F0C426801F1D3
:1013C00008040EFA04F434EA06070BD18F000CFA75
:1013D00007F822EA080205FA07F7282B42EA070273
:1013E0000AD1446101310829E9D14260BDE8F081A8
:1013F000482B08BF0761D6E7482B08BF0461F1E717
:101400004FF6FF730380022383700423C370704779
:101410008368194214BF012000207047806880B2A1
:101420007047C06880B27047416170470AB101617E
:10143000704741617047C160704741F480338361F8
:101440008161836183698369704700000028164ABF
:1014500030B500F44015B4BFD3695368B5F5401FEB
:1014600084B210D1556823F0706325F07065556023
:1014700019B1420D1201944023430B4A0028B4BF16
:10148000D361536030BDC2024DBF0322420D120131
:10149000C0F303454CBFAA4004FA02F223EA020358
:1014A00043F07063E4E700BF0000014010B50F2473
:1014B00001F0030301F0FC0101F1804101F58031ED
:1014C0008A689B009C4022EA04028A608A689840ED
:1014D0001043886010BD0000034A536823F0F003F6
:1014E00018435060704700BF00100240034A536821
:1014F00023F4E06318435060704700BF00100240BF
:10150000034A536823F4605343EAC00050607047B5
:1015100000100240014B1860704700BFD8004242E3
:101520001C4A10B5536803F00C03042B01D0082BA0
:101530001FD0194B03605368184CC3F30313E15CCD
:101540000368CB4043605168C1F30221615C23FA18
:1015500001F181605168C1F3C221615CCB40C3607D
:1015600052680F49C2F381328A5CB3FBF2F3036124
:1015700010BD53685168C3F38343CC0303F10203E6
:1015800002D408494B43D5E751688903F9D402498D
:10159000F8E700BF0010024000127A0004000020AB
:1015A0000000002000093D00044B9A6911B110436E
:1015B0009861704722EA0000FAE700BF001002407D
:1015C000044BDA6911B11043D861704722EA000078
:1015D000FAE700BF00100240224A038890429BB203
:1015E00012D002F5006290420ED0B0F1804F0BD0C5
:1015F000A2F59832904207D002F58062904203D063
:1016000002F58062904203D14A8823F070031343AD
:10161000154A904208D002F5806290421FBF23F421
:101620004073CA889BB2134303808B8883850B88E1
:1016300003850C4B98420FD003F5006398420BD002
:1016400003F54063984207D003F58063984203D0C6
:1016500003F58063984201D10B7A038601238382CC
:10166000704700BF002C014000100040038C70B593
:1016700023F480531B041B0C0384038C8488828B0B
:101680000D8822F4E6421204120C42EA052223F4E9
:1016900000530D894E881B0435431B0C43EA053368
:1016A0000B4DA4B2A84292B29BB203D005F50065DF
:1016B000A84205D18D8924F4804444EA8514A4B25B
:1016C00084808283CA88A0F84020038470BD00BF54
:1016D000002C0140038821B19BB243F00103038039
:1016E000704723F001031B041B0CF8E783899BB2AE
:1016F00012B119438181704723EA0101FAE7FFF72C
:10170000F5BF038923F007031B041B0C03817047FB
:10171000038821B19BB243F080030380704723F01C
:1017200080031B041B0CF8E7838B23F400631B046A
:101730001B0C43EA012189B281837047038923F09E
:1017400080031B041B0C038103899BB21943018195
:101750007047A0F840107047C94389B201827047B2
:1017600030B50D460446038A8A899BB2C98823F4A2
:1017700040530B4303828389A98823F4B05323F099
:101780000C031B041B0C0B43298987B00B4369898D
:101790000B439BB28381838A9BB223F44073134330
:1017A000838201A8FFF7BCFE174A039B0499944269
:1017B00018BF19461922A3894A4313F4004F2B6816
:1017C0004FF0640514BF5B009B00B2FBF3F1B1FB6B
:1017D000F5F3A2891801120405FB13130BD5DA00E7
:1017E0003232B2FBF5F202F0070242EA00039BB28A
:1017F000238107B030BD1B013233B3FBF5F303F097
:101800000F030343F3E700BF00380140838921B190
:101810009BB243F400538381704723F400531B04AD
:101820001B0CF8E701F01F0310B5C1F342140121AE
:10183000012C01FA03F105D10C3003683AB11943C8
:10184000016010BD022C0CBF10301430F5E723EA04
:101850000101F5E7C1F3080181807047038819424F
:1018600014BF01200020704710B50748FFF7D9FDCD
:10187000C0F3C0040448FFF7D4FDC30648BF44F0DA
:101880000204204610BD00BF000C014010B5064CFC
:10189000002220460821FFF7C9FD2046BDE8104080
:1018A00000221021FFF7C2BD000C014037B5012115
:1018B0000820FFF779FE02238DF806301823102543
:1018C0000B4C02A921F8043D20468DF80750FFF784
:1018D00045FD204600220821FFF7A8FD00222946E9
:1018E0002046FFF7A3FDFFF7D1FF03B030BD00BFD7
:1018F000000C014038B50C4C0546627822B920B97D
:10190000FFF7C4FF0023E37238BD420604D501226D
:1019100008210648FFF78AFD2B06F3D50122102186
:101920000248FFF783FDEDE7880D0020000C014021
:1019300010B5064B04461B78022B06D002F0C4FEFD
:101940002046BDE81040FFF7D5BF10BD880D002030
:101950002DE9F0411148FFF7E1FC04281AD14FF6B8
:10196000FF760E4DDFF844800D4F35F808100D4B13
:10197000B1422B4410D0FC182846FFF7B3FC234695
:101980001988B14202D0A81CFFF7ACFC064B043505
:101990009D42EAD1BDE8F0813B44F1E700FC01083B
:1019A000C60800200204FEF700000208C60CFE175D
:1019B0000C4A30B510460C4B0C4C1D7803F17841A5
:1019C0000133A1F5FE31A3425554F6D113780A2B09
:1019D00006D00023FF22C2540133B3F5806FFAD141
:1019E00030BD00BFC608002000FC0108000002084E
:1019F000014B185C704700BFC6080020014B19540A
:101A0000704700BFC60800200023F0B40A4C451EF2
:101A100025448F18B94204D120448354F0BCFFF709
:101A200097BF3BB9DB0911F8016B3344DBB205F812
:101A3000016FEFE70123F6E7C60800200023F0B5A9
:101A40000B4C4D1E25448718B84205D12144885CB3
:101A5000C31A58425841F0BD15F8016F2BB9DB0984
:101A60003344DBB200F8016BEEE70123F8E700BF77
:101A7000C608002008B500216022074806F0B5FE20
:101A80000649002003F09FFE20B9BDE8084007206A
:101A900002F04ABF08BD00BFC80C0020FC0C0020AB
:101AA0000149024805F07ABABC0D0020E80C00207C
:101AB0002DE9F04F5C2299B081460021A54806F03F
:101AC00094FEA54BA54A984603F108051C4603CC95
:101AD000AC4210605160234602F10802F6D1206842
:101AE000002510602379137199F80030242B40F001
:101AF0005D870123974A9570537003221D468DF828
:101B00003B20002426460994089406949DF83B3017
:101B100019F803B0BBF1000F1ED126B1069B002BB4
:101B200008BF02230693A10605D58A4BDA6A8C4BBF
:101B30009A4200F32087EA0740F1E081E30740F191
:101B40002387844FFB78012B40F0E6813869854973
:101B5000FFF7ECF83861DFE1ABF1410A5FFA8AF296
:101B6000192A00F2F68601330FAA0DF13B0148460F
:101B70008DF83B3001F006FD002800F0ED860F9B4C
:101B80001846079306F098FFFFF7D2FAC7B2384617
:101B9000FFF778F8079B01461846FEF7BDFF72492C
:101BA000FFF7C4F806F05CFFBBF1470F82B222D00A
:101BB000BBF14D0F00F0DC80BAF1190F4AD8DFE815
:101BC0001AF0170134014900490049003B0149005E
:101BD00049004001490152015B014900600149008F
:101BE00067016C01710175017A01490049004900E2
:101BF00088018F019601282F00F0A58032D8132F7D
:101C000023D8112F79D2042F09D06FD30A2F21D1D5
:101C10002AB9069B002B40F0A286012306934D4B68
:101C200007F0FD011C291F7002D05C2F40F08D8051
:101C30000AB10A2A0ED1384418700023099A1A41B1
:101C4000D20740F1CD8015255EE01C2FE0D003D8EF
:101C5000152F69D9142557E0212F47D0262F45D0BD
:101C60001E2FD4E73D2F6AD01BD8352FD7D011D8DF
:101C70002B2F01D0312FEDD1069B002B40F06F862A
:101C8000312F57D1334B9DF818209A710322082326
:101C90000692D3E73B2FDDD82E4B363FDF71092369
:101CA0002FE05B2F18D85A2F32D2502FD2D129498A
:101CB000262F4F704BD1A2F114039BB21E2BC9D813
:101CC0002A4820FA03F3D807C4D50A23B2FBF3F25B
:101CD000763A4A700123B1E75C2F99D05E2FB9D8CC
:101CE0001C4BC7F15E079F7005230AE0069B002B83
:101CF00040F0358602230693D9E7164B113F5F71FA
:101D00000223002A9AD01725284619B0BDE8F08F83
:101D100022B9104B5A3F1F7103238FE70A2A99D12A
:101D20005A2F97D0042389E70A4BC7F11507DF70B4
:101D30000623E6E70A2A8DD10122064BA5E7002AF1
:101D400088D10A237AE70723DBE70023D9E70123B9
:101D5000D7E700BF280D0020C80C0020290D002067
:101D6000809698003333CB410000C84201041040F4
:101D7000002AC8D1052F0AD8032F1BD3042FA94B43
:101D800021D0052F21D010229A720C2356E7092F5B
:101D90000AD8072FA34B1AD3082F1DD0092F1DD007
:101DA00080225A720D2349E71E2F7FF453AF9D4BBB
:101DB0001F7202E01FB1012FF9D10B233EE703226E
:101DC000984B1A72F9E72022DEE70022DCE70422B2
:101DD00045F48075DA72D8E74022E2E70022E0E7B6
:101DE000012202FA03F3099A13439BB209938DE689
:101DF0000D270F9A8B4B46F008065A6544FA07F3F5
:101E0000DB0700F1B28540F261333B41D80706D5CC
:101E100000210F98FFF728F9002840F0A985012339
:101E200003FA07F73C43A4B270E60F9A7D4B46F0E5
:101E300010069A650E27E1E70F9A7A4B00271A6180
:101E4000DCE7784B0F9A01275A61089B43F00103A6
:101E50000893D3E7734B0F9A02279A61089B43F0CC
:101E600002030893CAE76F4B0F9A0327DA61089BB6
:101E700043F004030893C1E76A4B83F828700427F2
:101E8000BCE70F98FFF72EF9664B0527D862B5E738
:101E90000F9A644B06271A63B0E70F9A614B5A6397
:101EA0000727ABE70F9A5F4BDA63F9E70F9A5D4BB1
:101EB00008271A64A2E75C490F98FFF7F3F8002897
:101EC00040F050850222574B83F844701A7309275B
:101ED00094E70F9A534B46F001069A640A278DE760
:101EE0000F9A504B46F00206DA640B2786E70F9AEA
:101EF0004C4B46F004061A650C277FE7494FBB7828
:101F0000012B18D1069B022B06D17B78502B03D0D6
:101F100013B1E70740F1388514F4807F08BFD8F883
:101F20001030404F08BF3B643B78042B11D1610651
:101F30000CD41C25E8E698F80130002BECD1E00722
:101F40003FF500AED8F814303B61E5E724F04004DB
:101F5000A4B27B79002B42D0012B0CBF01230023BC
:101F60000C930CBF002302230B930CBF022301230D
:101F70000A93FB78012B37D0069B032B05D1BB7945
:101F8000012B02D1042E40F0F984DFF8A4E013AF56
:101F9000BEE80F000FC7DEF800303B60099B214F01
:101FA00013F4007F39D197F800A0BAF10A0F50D08E
:101FB000BAF15C0F00F0EF80069B032B40F020810C
:101FC000BAF11E0F00F05C81BAF1350F00F0738199
:101FD000BAF11C0F40F00C811449062052E1022294
:101FE0000C9201220B92C3E74FF00009DFF844A0E6
:101FF000DFF844B046FA09F3DA0706D5DAF800004C
:102000005946FEF793FECAF8000009F10109B9F13B
:10201000050F0AF1040AEDD1AEE7F87906280DD9CB
:102020001D2571E6280D002000007F433C0D002097
:10203000FC0C0020700D00203333CB4198F80630A3
:102040008342B0D013A903F0BEFB0028ABD1072513
:102050005AE60EB91A2557E614F0500F3FF469AF4F
:10206000386B06F029FDFFF763F8C0B20628D7D811
:1020700097F82830142B05D0022B7FF4EBAD230604
:102080003FF5E8AD24F05004A4B200287CD001381C
:10209000C3B20793A749079803F095FB0028D6D051
:1020A0004FF0000B97F82830DFF888A2A24F0D936D
:1020B000D7F85C80AAF11409203746FA0BF3D90748
:1020C00014D50D9B142B61D1B96A3868FEF724FD35
:1020D000DAF83410FEF720FDBBF1020FCAF8000059
:1020E00004D14146FEF718FDC9F81C000BF1010BA5
:1020F000BBF1050F0AF1040A07F10407DDD18F4B8C
:102100005F789A46502F40F0DC80002E40F03984F2
:1021100015F00103069A15BF24F0210424F4487435
:10212000A4B224F0010412B124F4F844A4B2002CA7
:1021300040F03684109411941294002B00F03882F1
:10214000099B23F04903002B40F02D847B4B1B7827
:10215000352B02D0002B40F02684774C7749236939
:10216000227A1193637A10A813438DF8483000F057
:102170002BFC054600287FF4C7AD714E20340FCEEE
:102180000FC433682360BFE5FB7982E7DAF83430A7
:10219000CAF80030AAE7002E3FF45CAF0027D8F859
:1021A0005C30DFF89CB1DFF89C8107930DF14C099E
:1021B000ABF1480A46FA07F2D2071CD559F82710A6
:1021C000D8F80000FEF7A8FCDBF80010FEF7A4FC2E
:1021D000022FCBF8000004D10799FEF79DFCCAF846
:1021E00050000137052F08F104080BF1040BE1D171
:1021F0000023079383E7D8F82820CBF80020F0E7E6
:10220000002E3FF4DDAE4FF0000B3B794C4F0793AF
:10221000494BA7F14809DA6D03F120080D9246FAFF
:102220000BF3DB070CD4D8F800303B600BF1010B4B
:10223000BBF1050F08F1040807F10407EFD1BFE671
:10224000BAF1350FF2D0079B9BB913ABD8F8281021
:1022500053F82B00FEF762FC3968FEF75FFCBBF118
:10226000020F3860E2D10D99FEF758FCC9F8500012
:10227000DCE73868D8F80010FEF750FC3860D5E786
:1022800007202C4903F09FFA00283FF4E0AE16B96E
:102290000796069633E700232849274846FA03F2B3
:1022A000D70704D49A0057180244126A7A6101339E
:1022B000052BF3D19CE7214B5B78012B98D91E2588
:1022C00022E5069A022A7FF423AF2FB91346002E87
:1022D00008BF002306931BE700211869FEF7BAFE2A
:1022E000002840F051838C2F12D009D8022F2BD018
:1022F000032F2BD0012F7FF40BAF002E069BE7E7B7
:102300008E2F05D002D38F2F7FF402AF45F010053A
:102310007237FFB2012F98BF45F00805002E3FF439
:1023200099AE14220649074806F050FA002842D018
:10233000EEE600BF3C0D0020C80C0020280D002058
:10234000700D0020E80C002045F00405002E3FF43D
:1023500081AE01230A9A03FA02F90B9A934049EAE3
:10236000030916EA090F00F012830A9B0A9ADFF8A4
:1023700034B2123308325BF822105AF82300FEF709
:10238000CBFB0B9B0B9A1233083207465BF82210EB
:102390005AF82300FEF7C0FB14F08003804600F0DB
:1023A0008F8024F0800414227A490BF12000A4B21B
:1023B00006F00CFA08B92125A6E49AF80330012B9F
:1023C00006D1DAF83C007449FEF7B0FCCAF83C00CC
:1023D000DFF8D4A14FF08141DAF83C904846FEF78F
:1023E000A5FC4946FEF7A2FC394681463846FEF771
:1023F0009DFC01464846FEF78FFB4146814640461C
:10240000FEF794FC01464846FEF786FB0021814614
:10241000FEF72AFE002840F0BD824846FDF7FCFF8B
:1024200006F05EFB834689463846414601F046F990
:10243000FDF7F2FF09F100490B46024649465846AE
:10244000FEF768F9FEF714FB9AF80130DFF858A19F
:10245000032BDAF83CB081464FF0000108BF00F1D1
:1024600000495846FEF700FE28B10BF1004B09F178
:102470000049CAF83CB00A9B4146484603F1040BA8
:10248000FEF754FC01463846FEF746FB4FF07C5100
:10249000FEF74CFC0B9B0AEB8B0B0433CBF80400D0
:1024A000394648460AEB830AFEF740FC4146FEF7F0
:1024B00035FB4FF07C51FEF739FCCAF8040027E6E3
:1024C000089A19EA020F00F068829AF8032024F0B3
:1024D0000E04012AA4B244D00B9BDFF8CCA003F178
:1024E00004090AEB8909D9F804104046FEF714FBE9
:1024F00083460A9B384603F104080AEB8808D8F89B
:102500000410FEF709FB594601F0D8F8D9F8041079
:102510000746D8F8040001F0D1F80146CAF83C009B
:1025200080463846FEF7F8FA20F000471B49384647
:10253000FEF7B8FD00283FF4EBAD4FF07C51384674
:10254000FEF7B0FD00287FF436AF15494046FEF790
:10255000EDFB01463846FEF7A5FD00287FF42BAFC2
:10256000D6E59946DFF844A0DFF82CB0089B43FA83
:1025700009F3D90706D5DAF800005946FEF7D6FB6D
:10258000CAF8000009F10109B9F1050F0AF1040ABE
:10259000ECD1A1E7700D00203333CB410AD7A33B28
:1025A0006F12833AC80C0020280D00203C0D00203B
:1025B000AC4BAD4CB3F86A30AC4F13F0020F0ED0F9
:1025C0007B78013B022B88BF45F04005002E00F0D0
:1025D000DD80069B022B40F0D98045F08005FB6A28
:1025E000E361BB78637013B108238DF848303B6911
:1025F000D7F840806361414620691093FEF72AFDB9
:1026000005F0400608B1AA060BD5607A38B12B0652
:1026100005D4002E00F0CE80002103F083FC3B6C3B
:1026200023610EB92369119397F84430B87A237661
:10263000637A834204D0119903F074FCBB7A63720D
:102640009DF84830627A787A13438DF84830237ABF
:10265000834206D0FFF76CF97B7A002B40F0AC8008
:1026600023729DF84830227AE80543EA02038DF888
:10267000483015D5F87AA37A834200F0A08004F0A0
:10268000A9FFFB7A012B1CBFA27A1343A3729DF80A
:102690004830A27A25F480751343ADB28DF84830E6
:1026A000387BE37A834200F0988004F0A3FF3B7B01
:1026B000002B40F08F80E3729DF84830E27A13439C
:1026C0008DF848303B78042B02D1386B00F092FE35
:1026D0007B792371FB78A370069B032B0DD1BB790B
:1026E00063710BB900233B653E6DE06D3146FEF72B
:1026F000B1FC10B9E66504F039FCFB79A2799A4285
:102700000BD05B4E0DF14C0EA371BEE80F000FC64F
:10271000DEF80030336004F029FC3B79E3703B784D
:10272000262B00F0998060D81C2B7BD01E2B79D0F3
:102730000A2B63D07B78502B23700FD0069A022A85
:102740000CD1012B40F0A88010A94A4800F070FC81
:10275000494D484E0FCE0FC533682B603D7AE57169
:10276000002D3FF4D1AA01F0AFFFE379032B434BD7
:1027700040F0C4801B78022B04D0082004F04EFCEB
:1027800001F038FE0025E571FFF7BEBA637A102B21
:102790007FF425AF2378013B022B05F0400305D8D9
:1027A000002B3FF41CAF45F0200518E7002B7FF409
:1027B00016AFF8E7414630E7227A134350E759074E
:1027C0007FF565AF184604F005FF0423A3720123CB
:1027D000FB725CE7E27A13436DE79A077FF56CAF13
:1027E000184604F007FF002365E75C2B4AD0662BF0
:1027F0004CD0282B9ED1204907202FE02049079854
:1028000002F0F4FEA379079A934293D1184EDFF8B1
:1028100070E0BEE80F000FC6DEF80030336004F051
:10282000A5FB87E79DF8483043F001038DF8483059
:10283000069B1BB110A90F4800F0FAFB10A9104825
:1028400000F0F6FB0C4EDFF838E0BEE80F000FC6D4
:10285000DEF8003033606DE70620074902F0C6FE5F
:1028600068E700BF50100020C80C0020280D002091
:10287000FC0C0020700D0020E80C0020880D0020CA
:102880003C0D00204B4EDFF838E1C2E71422002156
:10289000484805F0AAFFC2E733B99DF8483043F035
:1028A00001038DF848304FE7023B012B12D80C9BF7
:1028B000C5F3800503930B9B049502930A9B3E4A44
:1028C0000193FB6B10A900933C4B03F1340000F023
:1028D000E3FB3DE79DF84830EAB243F0040310A95A
:1028E00037488DF8483000F0BDFD00283FF430AF88
:1028F00001287FF433AFFFF7D3F82FE764220025D8
:102900000126DA711A725A721B782670022B257111
:10291000E5706570A57165722572A67215D029499A
:10292000284602F050FF00283FF491AB04F01EFB54
:102930000021284603F0B4FA2846FEF7DBFF3046B4
:1029400004F02AFE284604F0FFFD082002F014F8E7
:1029500018E70125FFF7D8B90225FFF7D5B91825E3
:10296000FFF7D2B92625FFF7CFB91925FFF7CCB964
:102970000425FFF7C9B91B25FFF7C6B92525FFF7C1
:10298000C3B91F25FFF7C0B91625FFF7BDB920252C
:10299000FFF7BAB92225FFF7B7B92325FFF7B4B976
:1029A0002425FFF7B1B91025FFF7AEB98DF83B50DC
:1029B000FFF7A7B8100D0020E80C00203C0D002008
:1029C000700D0020FC0C002038B50B690546036033
:1029D000037A01F1480443F004030372104BB3F887
:1029E0006A3013F0200F10D129460E4D204600F01A
:1029F0001FFB2C7884B900F0CFFF68B120232B7027
:102A000003F060FD03F0CAFA07E0204604F0D4FAB0
:102A10000028E9D00F2400E00024204638BD00BF84
:102A200050100020880D002004F0BCB94FF48072D3
:102A3000014BC3F88420704700E100E038B510482E
:102A4000FEF7ECFC03460F4AB2F86A2052065CBF60
:102A500080F47C439BB28BB10022012410460A49CA
:102A600051F822502B421CBF04FA02F5284302F110
:102A7000010218BFC0B2052AF2D138BD184638BDD0
:102A8000000C0140501000204CA6000810B54FF477
:102A90008060FEF7DFFB18B14FF48060FEF7E8FBC3
:102AA0004FF48050FEF7D6FB18B14FF48050FEF77C
:102AB000DFFB4FF40060FEF7CDFB18B14FF4006070
:102AC000FEF7D6FB4FF40050FEF7C4FB18B14FF4ED
:102AD0000050FEF7CDFB4FF48040FEF7BBFB18B172
:102AE0004FF48040FEF7C4FB144BB3F86A30DB05AB
:102AF00014D400244FF48072114BC3F88421114B7D
:102B00001B78012B18D0104B1B78ABB900F010FDCF
:102B100084B10A20BDE8104004F00EBC4FF4004020
:102B2000FEF798FB0028E4D04FF40040FEF7A0FB2E
:102B30000124DFE70120EDE710BD00BF50100020A9
:102B400000E100E0880D0020D00D00202DE9F04FBD
:102B5000744B8FB05C7882469846002C40F0A88079
:102B600006234FF00009704D704E714F0894069483
:102B700007948DF8203055F8242004A90A554AFA04
:102B800004F2D0074FEA84030AD533443946D86BA0
:102B9000FEF7CCF849468346FEF766FA00B9D946F7
:102BA0000134052CE7D104230127604D0193D5F8AA
:102BB00074B009AB18465F49039304F0EFF90020A5
:102BC0000646014695F86C3009F1004E0293039BCE
:102BD0004AFA01FC1CF0010F18D00024554A0130BC
:102BE00042F82140029AC0B242FA01FC1CF0010FE7
:102BF00003D027B143F821E003E0002FFAD043F8D7
:102C0000219004AA12F801C046EA0C0601310529F8
:102C1000DED1FEF733F805F0B7FF88F8066001460D
:102C20005846FEF783F806A9069009A800F060FF51
:102C3000042388F8043003F045FC03F0AFF9DFF813
:102C4000009187B1FFF7FAFE002304AAD25C32425A
:102C500004D040FA03F1C90748BF96430133052B5E
:102C6000F3D188F8066003F02DFC99F8003013F0DA
:102C7000340F4BD099F80060F6B2F30602D5062067
:102C800004F05AFBB40602D5072004F055FB002FD0
:102C900044D1FFF7D3FE1AEA000F02D0082004F057
:102CA0004BFB254B1B7833B100F042FC01F0A2FB3B
:102CB0000FB0BDE8F08F042004F034FB03F096FB66
:102CC000B5F8780000F0F0FC87F001060FBB1B4957
:102CD000E86FFEF72BF88146D5F870B0019B3746B8
:102CE0005C1E14F0FF0301937FF463AF1C46224681
:102CF000104B4AFA04F1C90748BF43F824200134B5
:102D0000052CF6D1002388F80430D1E7F00698D1DD
:102D1000D4E7D5F87C90D5F874B0DFE77307C0D559
:102D20000920BCE7880D002060A600085010002094
:102D30000000C0BFBC0D0020D00D00200000A0404E
:102D4000A50D002010B504F037F9C0B101220C4CDC
:102D50002078E270082808D000F0EAFB022004F096
:102D6000EBFABDE8104001F045BB04F057F901F063
:102D700041FB63781BB92378002BF8D1ECE710BD39
:102D8000880D0020F0B5074687B04FF44070FEF77D
:102D9000EFF900240125252301A88DF804308DF8D2
:102DA00005408DF80750FEF7EDF9294644F205007D
:102DB000FEF7FAFB4FF40073ADF8003018238DF8DE
:102DC00003300323194E694630468DF80230FEF772
:102DD000C5FA4FF48063ADF80030042369463046ED
:102DE0008DF80330FEF7BAFA0C23ADF80C40ADF8BD
:102DF0000E40ADF81040ADF814400D4CADF8123057
:102E0000A38902979BB243F00C03A38102A9204639
:102E1000FEF7A6FC2A46204640F22551FEF702FDA9
:102E200029462046FEF7F2FC07B0F0BD000801403D
:102E3000003801404FF47A72074B5A6000229A60C2
:102E400001221A601A6802F00112012AFAD0002247
:102E50001A609A60704700BF10E000E010B5074CA0
:102E60004FF4005122780648FEF7E0FA237813F178
:102E7000FF3318BF0123237010BD00BF14000020D2
:102E8000001001402DE9F34101215848FEF7DEFA18
:102E9000574A00209369574E43F0010393614FF066
:102EA0008062554B00245A60FEF716FB4FF4806099
:102EB000FEF71CFB0020FEF723FB01211020FEF78C
:102EC00073FB02238DF8063010238DF807304FF482
:102ED0000053374602A921F8043D4848FEF73EFA60
:102EE0004FF4E130FFF74EFF05F008FA05F011FA54
:102EF00004F0A0FFFEF7CEF9FEF75AFD404ADFF8D6
:102F0000FC80136823F00403136002F0A5F902F0BB
:102F1000CDFD03F0EFFE03F045FF002002F0F2FDCF
:102F200014220021374805F060FC34701C22002177
:102F30003846357805F059FC6423142200213248C4
:102F40003570F3713372737205F04FFC2F4B304DB7
:102F50001C70304B1C70304B1C70304B1C70304B55
:102F60001C70304B1C70304B1C7002F01FFBFEF7C6
:102F700081FD95F8800002F0C5FD95F8800002F013
:102F800095FD04F099FAFEF791FC03F00BFF01F0B8
:102F90003DF800F0D1FC03F029FA00F00DFFFEF738
:102FA0007FFD4FF480414046FEF732FA012812D0EF
:102FB0001E4D10212846FEF751FC80B94FF4FA70DF
:102FC00000F072FBFFF74AFFF3E740F2DC5000F03D
:102FD0006BFBFFF743FF05F0A3FB0028F5D001F0E2
:102FE0000FFDFFF73BFF01F0DBFA9FE70004300025
:102FF00000100240880D0020000001400010014038
:1030000010E000E0BC0D0020A80D0020A60D00205F
:1030100050100020D10D0020840D0020A50D0020AF
:10302000D00D0020850D0020A40D002000380140A7
:10303000F8B5174C0746B4F86A200D4612F0200F79
:10304000144E04D03378202B01D0FFF77BFE337869
:10305000022B1BD001F0CEF97378BBB900F0C6FC8F
:1030600010B101F009F8F5E72946384600F040FDB7
:1030700060B9B4F86A309A0708D52B7ADB0605D513
:1030800069681020BDE8F84002F04CBFF8BD00BFF1
:1030900050100020880D00202DE9F04F1C4692466C
:1030A0008FB09DF86C309DF8645003939DF870309C
:1030B00054F825700693AB001A440290E31801916E
:1030C00038465AF8251008920993FDF727FD9DF818
:1030D000688004904FEA88030AEB0302E31854F86F
:1030E00028405AF8281020460A920B93FDF716FD47
:1030F000029B0499059053F82500FDF70DFD029BF6
:103100000546059953F82800FDF706FD07F100472D
:10311000834629463846FDF709FE04F100448046FF
:1031200059462046FDF702FE01464046FDF7F6FCF3
:10313000FDF772F98046894638465946FDF7F6FD97
:10314000294683462046FDF7F1FD01465846FDF726
:10315000E3FCFDF761F94B464246189E05F0BEFCC4
:10316000FDF786FC069B0546002B45D0FDF754F97C
:1031700097A3D3E9002380468946FDF727FC48B191
:1031800095A3D3E9002340464946FCF7E5FFFDF748
:103190006FFC0546944B3146D3F85C803046FDF712
:1031A000BDFC4146FDF7B8FC4146FDF7BFFDFDF70C
:1031B00033F905F095FC8046894628464FF07C514E
:1031C000FDF7B4FD3146FDF7B1FD20F00040FDF7FD
:1031D00023F942464B46FDF79DFAFDF749FC05F001
:1031E000FFFBFDF7A5FF86B2CEB9019902980FB09B
:1031F000BDE8F04FFFF71CBFFDF70EF978A3D3E948
:10320000002380468946FDF7D7FB0028C2D072A371
:10321000D3E9002340464946FCF7A0FFB7E7019BEE
:1032200093F8088018F0080F0DD03046FDF72AFDFE
:10323000019B01461868FDF779FD019B28F00808FD
:10324000186083F808803046FDF71CFD8046014673
:103250002846FDF71FFE039B039A0AEB83030693A0
:10326000039B05465AF82310029B4FF0010B53F8BD
:103270002200FDF751FC4146FDF70CFE29460C905B
:103280002846FDF753FD01464FF08040FDF744FC12
:10329000564980462846FDF749FD4FF08141814659
:1032A0004046FDF73BFC01464846FDF73FFD4FF029
:1032B0007C5103904046FDF739FD4FF00008079020
:1032C0001FFA8BF39E4290D9B8F10B0F40D80399A7
:1032D0003846FDF72BFD079981462046FDF726FD70
:1032E00001464846FDF71AFC079981463846FDF726
:1032F0001DFD039907462046FDF718FD0146384697
:10330000FDF70AFC4C46074608F101085FFA88F809
:1033100004993846FDF702FC089B05991860204681
:10332000FDF7FCFB0A9B0C991860069B0BF1010B47
:103330001868FDF7F3FB069B019918605046FFF7EC
:1033400077FE2B4B5B78002BBAD00FB0BDE8F08F27
:103350005846FDF797FC2946FDF7E8FCFDF75CF8B9
:103360008046894605F04AFAFDF782FB4946044645
:10337000404605F0BBFAFDF77BFB099B0B9A1B68E7
:10338000814603F1004319462046D2F800800D9390
:10339000FDF7CCFC414607464846FDF7C7FC014611
:1033A0003846FDF7BBFB0D9B074619464846FDF71F
:1033B000BDFC414681462046FDF7B8FC0146484623
:1033C000FDF7AAFB4FF000080446A1E7AFF3008029
:1033D0008DEDB5A0F7C6A0BE182D4454FB211940B1
:1033E0008DEDB5A0F7C6A03E50100020ABAA2A3E36
:1033F000880D002010B5074B04461B78022B07D020
:1034000001F062F92046BDE81040002100F02AB921
:1034100010BD00BF880D002010B50446FFF706FB65
:10342000B4B12046FFF792FB00F0E4FF0B4B5B7852
:103430006BB9FEF735FB00F0BFFC4FF4F840FDF729
:1034400017FF4FF48072064BC3F884215A6010BDF9
:103450000420FFF77BFB0320E4E700BF880D00207A
:1034600000E100E02DE9F8432D4C0646237889461B
:10347000022B9046274650D001F026F9657815B109
:103480000220BDE8F883C8F3C000657100F0AAFD12
:1034900000F0C6FD40B1042003F04EFF00F0AAFF8B
:1034A000284600F09FFDEBE730464946FFF7C0FD98
:1034B00001231C4E0220337003F0B0FD00F09AFF90
:1034C0007B78002BDCD13B78002BF7D13378012BB4
:1034D00020D118F0100F19D0134C144D0FCD0FC47C
:1034E0002B6823600020307000F07CFD00F082FF2C
:1034F00002F07CFF00F020FA00F05EFC01F096FB89
:103500007879003018BF0120BDE8F883052003F06A
:1035100013FFE7E701237B71E4E70020BDE8F883B0
:10352000880D0020A60D0020A80D0020BC0D002055
:1035300008B5114B1B78DB061DD4102003F06EFD7F
:1035400002F0D0FAFEF7A2F90C4A137813F02C0F10
:1035500003D1127912F0060F0DD0042B09D1084BBC
:103560001B7813B9062003F0E7FEBDE8084002F01F
:1035700053BD0320F7E708BDA50D0020880D0020EE
:10358000D00D00202DE9F84F0B789146C218C35C8E
:1035900006462D2B884618D101275378951C00210B
:1035A0000A460C460846303BDBB2092B19D80132DB
:1035B000D2B2082A10D809B1013C64B200EB8000F5
:1035C00003EB400015F8013BEDE72B2B12BF551C18
:1035D000951C53780027E2E70029F3D1013464B247
:1035E000F0E7FE2B02D109B90121EBE7D2B1FDF7DB
:1035F00045FB00218246FDF72DFD48B9DFF85CB0A0
:10360000631C12DB19D150461349FDF78FFB82462C
:103610000FB10AF1004A0122AD1B013DC9F800A01B
:1036200088F800501046BDE8F88F50465946FDF71F
:103630007DFB0234824664B2E2E7002CE8D0DFF87A
:1036400020B050465946FDF771FB013CE3B282467B
:103650005CB2002BF5D1DBE7CDCCCC3D0AD7233CC7
:103660000000204170B50E460D49FDF75FFB05F0E7
:1036700077F9FDF75DFD0B4D84B27CB16B786BB9CA
:103680003EB900F0B7FE3220013CFFF7D3FBA4B2F5
:10369000F3E700F0FBFCAB789B07F4D570BD00BFEF
:1036A0000000A041880D002010B5044604B910BDEB
:1036B0000120013CFFF7BEFBA4B2F7E738B50D4689
:1036C0000146FDF733FB294604462846FDF72EFB4D
:1036D00001462046FDF722FAFCF79EFE05F000FAAF
:1036E000FDF7C6F938BD2DE9F8430026041F25462D
:1036F000B14600F1100755F8048F49464046FDF7E2
:10370000A9FC40B941464046FDF710FB0146304652
:10371000FDF704FA0646BD42EDD1304605F034FA15
:10372000014606464FF07E50FDF7B4FB0746616840
:103730003846FDF7FBFA44F8040FAC42F7D13046A7
:10374000BDE8F8832DE9F8430746884600244FF08A
:1037500000090D4D58F8246049463046FDF77AFCC3
:1037600060B9314657F82400FDF794FB20F000467D
:1037700029463046FDF796FC00B935460134052C44
:10378000E8D12846BDE8F883FFFF7F7F013010B500
:10379000C4B20C2C04D901F0CDFB102C08BF0024BE
:1037A000204610BD2DE9F74F554F564E97F8008033
:1037B00096F80090B8F1000F08BF4FF0100808F11C
:1037C000FF385FFA88F8C145019767D03C244E4D19
:1037D00004FB085BDBF82410DBF820A00846FDF7AB
:1037E0009DF9DBF82810FDF7A1FA83460146504603
:1037F000FDF73AFC00B9DA46B8F1000F14BF4346B2
:10380000102304FB0854013BDFB2B945C4F81CA0E7
:1038100032D04FF03C093278BA4233D0002FBA464A
:1038200009FB075B08BF10277B1EDFB2374B1A78F6
:10383000BA4201D102F030FE09FB0A5ADAF82080C0
:10384000DAF81C004146FDF705FC98B9DAF82410B7
:103850000846FDF763F9DAF82810FDF767FAE16921
:10386000FDF75CF9044601464046FDF71BFCC0B17C
:10387000CAF81C405C46CEE7244B1B784B4501D16F
:1038800002F00AFE4FF03C08307808FB0057FFF7C3
:103890007DFF0446019B1A78A24205D103B0BDE822
:1038A000F08FCAF81C80E5E708FB0459D7F81CB074
:1038B000D9F81CA058465146FDF7D6FB90B1796A5D
:1038C0000846FDF72BF9B96AFDF730FA5946FDF7BE
:1038D00025F9834601465046FDF7E4FB10B1C9F8CF
:1038E0001CB0347008FB0453196AD869FDF7B2FBA9
:1038F00000B134702046FFF749FF4F460446C9E740
:10390000D4050020D505002014020020D605002093
:1039100000230121044A1370044A1370044A1170F1
:10392000044A1370704700BFD6050020D40500205C
:10393000D7050020D505002008B52C22002103481A
:1039400004F053FFBDE80840FFF7E2BFD8050020B0
:1039500010B5084B084C1B782078834208D0FFF73D
:1039600015FF064B21781A782070914208BF187015
:1039700010BD00BFD4050020D6050020D5050020CD
:103980003C20034B1A78034B00FB0230704700BF0A
:10399000D405002014020020054B1878054B1B7835
:1039A00083421DBF3C22044B02FB003000207047C5
:1039B000D6050020D40500201402002008B5084BCD
:1039C0001878FFF7E3FE074B1B7883421FBF3C22AA
:1039D000054B02FB0030C06908BF002008BD00BFD6
:1039E000D6050020D405002014020020034B1878CF
:1039F000034B1B78C31A584258417047D605002024
:103A0000D705002038B5837E0546DA07446B15D507
:103A1000164B187AFDF736F91549FDF787F9014677
:103A20002046FDF783F904464FF07E512046FDF70E
:103A300039FB08B94FF07E54204638BD5B070BD4E4
:103A40000A4BD879FDF71EF90949FDF76FF90146D0
:103A50002046FDF76BF904462D6B20462946FDF7FD
:103A600021FB0028E0D02C46DEE700BF880D0020B7
:103A70000AD7233C2DE9F843184B194E1C78DFF880
:103A80006C80184F98F80030A34203D1164B9E6209
:103A9000BDE8F8833C2505FB04752846FFF7B2FF17
:103AA000814601463046FDF7DFFAA0B13146304687
:103AB000FDF73CF928623C2505FB0475EE6A286A8F
:103AC0003146FDF7EFFA00B12E622046FFF75EFEA9
:103AD0004E460446D6E749464846E9E7D605002063
:103AE000FFFF7F7F14020020D8050020D4050020AE
:103AF0003C222DE9F04F8A46A14CA24E257899B080
:103B000002FB056901900021484604F06EFE9AF818
:103B10000830DAF8042013F0020F14BF9A4F9B4FBD
:103B2000009489F81A30C9F8382009AC0FCF0FC4B7
:103B30003B68002723603C2303FB056B019BDFF8F8
:103B4000748253F8270058F82710FDF7EFF8FCF7B8
:103B500063FC04F089FE09A951F8271004AB43F86F
:103B60002700401A80EAE074A4EBE07449F827408B
:103B7000DBF8141023468C4238BF0B46CBF81430C8
:103B80000393FDF77FF858F82710FDF783F90EAC83
:103B900044F827000021FDF767FACDF80880039B61
:103BA00038B17B4ABBF8181052F827200A43ABF80B
:103BB00018200137052FC1D1002B00F0DD804FF018
:103BC0003C082046FFF78FFD08FB05682146C8F832
:103BD00028007048FFF7B6FD2146C8F824006E485B
:103BE000FFF7B0FD98F81A70C8F83000F9074FD504
:103BF000C8F83400009B4FF0000A1A78674B1B7816
:103C00009A4202D017F002074DD03C2303FB056314
:103C1000C3F81CA0C3F82CA03C2707FB0567BB7E9C
:103C20009B0733D44846FFF7EDFEDFF860818146FD
:103C3000D8F828A05146FDF735FA002800F0998001
:103C400051465046FDF772F83C2303FB0565EE6ACA
:103C500038623146286AFDF725FA00B12E62504DD0
:103C60000FCCC8F828900FC523682C4604AD44F843
:103C700024390FCD0FC42B6823604A4C009B207859
:103C80001870FFF783FD2070FFF78CFD012074E0B2
:103C9000DAF800103A07C8F83410ABD5D8F8280085
:103CA000FDF744F8A4E7D0460DF14C0B374B3B44ED
:103CB0005A69E3591046194603930192FDF736F805
:103CC00001464046FCF728FF019A039B80461146B7
:103CD0001846FCF721FF4BF807000437142FE5D1F5
:103CE00031494046FDF7DEF918B13C2303FB05637B
:103CF00090E72E494046FDF7B7F928B13C2303FB76
:103D000005632B4ADA6287E75846FFF7ECFC594611
:103D10002048FFF717FD414682464FF07E50FCF7E2
:103D2000FBFE4FF07C51FDF701F8FCF775FB04F04A
:103D3000D7FEFCF79DFE0746029B5046996DFCF7A7
:103D4000F5FF3946FCF7F2FF394680464FF07E50CA
:103D5000FCF7E2FE01464046FDF79CF800210746CD
:103D6000FDF782F900B100273C2303FB0563DF6206
:103D700052E74946484665E7184619B0BDE8F08F56
:103D8000D405002014020020BC0D0020D80500201E
:103D900038A600087810002064100020D605002006
:103DA000EC050020D7050020EFFF7F3FEFFF7FBF2E
:103DB000FFFF7F7F501000200023054A054850F880
:103DC000231042F823100133052BF8D1704700BFB0
:103DD000D8050020BC0D0020064B1A78064B1B7836
:103DE0009A422CBF03F10F0003F1FF30801AC0B2DA
:103DF000704700BFD4050020D605002008B502F0AA
:103E00004BFB044B1A78044B1A70BDE80840FFF7CF
:103E1000C9BC00BFD6050020D505002010B5441E42
:103E200014F8010F00B910BD01F02EFAF8E763286D
:103E300038B51DD90A24B0FBF4F304FB1304303465
:103E4000E4B2D8B20A25B0FBF5F305FB1305303513
:103E5000EDB2D8B23030C0B201F016FA15B1284632
:103E600001F012FA54B12046BDE8384001F00CBA16
:103E700009284FF00004E5D82546EBE738BD30B5FA
:103E800085B028B9302005B0BDE8304001F0FCB95C
:103E900000230A2104AA5C1C1344B0FBF1F201FBCD
:103EA0001200E4B203F80C0C23461046002AF1D1AC
:103EB00001AA15190CB905B030BD15F8010D013C6A
:103EC0003030C0B201F0E0F9E4B2F3E7F0B50D46EE
:103ED00085B000210446FDF7C7F820B12D2001F080
:103EE000D3F904F100442E46284F012E2AD86B083E
:103EF000C3EBC31305EB430313F0FF0F04D02046BD
:103F00002349FCF713FF04464FF07C512046FCF791
:103F100005FEFDF7E7F800230A22DCB20133C8B939
:103F20003022631E6B44AC421FD306D104AA631C2B
:103F30001444302204F8102CDCB20DEB0406CCB98A
:103F400005B0F0BD20463946FCF7F0FE023E0446BF
:103F5000F6B2CAE704A90C44B0FBF2F102FB11006F
:103F6000303004F8100C0846D7E70134E4B203F807
:103F7000012FD8E7AC4202D12E2001F085F916F8C6
:103F8000010D013C01F080F9E4B2D8E70000C8421D
:103F90000000204108B5074BB3F86A30DB0707D5AE
:103FA0000549FCF7C3FE0421BDE80840FFF78EBFBA
:103FB0000321F9E7501000208B42213D08B5074B43
:103FC000B3F86A1011F0010103D00549FCF7AEFE09
:103FD0000121BDE80840FFF779BF00BF5010002065
:103FE0008B42213D0022074B1A70074AB2F86A2023
:103FF00012065CBF01221A7018B11A7882F0010211
:104000001A707047D20D00205010002008B508200B
:104010000121FDF7C9FABDE808400020FFF7E2BF23
:1040200008B50548FDF7FAF9044B00F001001B78CC
:10403000181A18BF012008BD000C0140D20D002045
:1040400038B5FFF7EDFF68B10022074B074C084D6C
:104050001A700FCD0FC42B68064A2360137843F003
:104060004003137038BD00BFA60D0020A80D00202E
:10407000BC0D0020A50D002008B5FFF78DFC20B178
:10408000BDE80840022002F0C9BF08BDF8B5384BB2
:10409000384C1B78384E03F0FF054BB101272846FA
:1040A000013D277000F056FCBD420CD903F04EF9DB
:1040B000337803F0FF05002B00F0BA80EF060CD533
:1040C00001236370F8BD384600F056FC102003F061
:1040D00029F93378DB06FCD5E8E7EE0704D500F0D4
:1040E00029FF012003F01EF915F0E8075AD02378C4
:1040F0006EB213F0030F47D113F0280F10D0A3783E
:1041000013F0C00F0CD102F0C7F9022323712378FA
:10411000202B05D1002E07DBA37863F07F03A3706B
:1041200023780BB90122A270680605D599065EBFF7
:10413000A27842F04002A2702A0704D513F0E00FE3
:1041400004BF10232370A8061ED5062000F014FC1F
:10415000A378190614D42278402A0FD11A0704D55F
:1041600023F01C0343F00203A3704023237007E0F5
:10417000D00D0020880D0020A50D0020802AF4D14C
:10418000A37843F02003A370002E08DA2378012BD4
:1041900002BFA37843F00503A37080232370384641
:1041A00003F0C0F8A80723D515F0680F1DD12378B8
:1041B000402B07D1A37813F0200203D1D90640F198
:1041C000D48022702378002B00F0D580DF060CD538
:1041D000A278D60709D5102B40F0CD80A37A002B0A
:1041E00000F0C98043F00803A372022003F09AF89C
:1041F00068071DD5237813F0D00F00F0D180E37845
:10420000002B40F0CD8094F90230002BC0F2C88022
:10421000FFF7F4FD2379990748BFA27823F006033E
:1042200044BF42F00102A2702371042003F07AF827
:104230006D4B1B7803F0FF05002B38D003F0A2F87C
:10424000E07915F0010F0CBF03466423AA0748BFAD
:104250000A336F0744BF0A3B9BB22E0744BF0133AA
:104260009BB2E90644BF03F1FF339BB2FF2B28BF8B
:10427000FF239BB20A2B38BF0A23217A15F0200FA7
:1042800014BF64220A4615F0400F18BF322215F001
:10429000800F18BF1922984201D18A4207D0E371DA
:1042A00000232272E372FFF7E5FBFFF7A7FD4F4BF8
:1042B0001B7803F0FF06002B4FD003F06BF8627AF7
:1042C00016F0010F0CBF13466423B70744BF0A332F
:1042D000DBB2750744BF0A3BDBB2300744BF013392
:1042E000DBB2F10644BF03F1FF33DBB2C82B28BFBA
:1042F000C8230A2B38BF0A239A4206D063720023D0
:104300002279E37242F008022271B70607D52378BA
:10431000102B04D1A37A002B5FD10223A37216F0D5
:10432000C00F1AD0237813B113F0180F15D0304FE7
:1043300030063D7A05D529064CBF05F07F0545F0CE
:104340008005720605D56B064CBF05F0BF0545F02C
:1043500040052846FDF7CEFA3D72237813F0FC0F96
:1043600040D0BDE8F84002F0ADB85A0744BF43F072
:104370000803A37026E700232371FFF70DFB58B154
:10438000A37813F0400307D1A3700823237002F031
:1043900099F801F003FE28E70023A370237024E7B7
:1043A00094F90230002B09DA00232371FFF7C4FAD5
:1043B00002F01CF8FDF774FBFFF7FEFCA37813F086
:1043C00020021FBF03F07F0343F00103A3704023CB
:1043D0000ABFA2702370227027E7DD079FD543F044
:1043E00004039BE7F8BD00BF850D0020A40D00204D
:1043F000C80C00202DE9F84F664CFFF747FEA37864
:10440000ABB1FFF7C9FAA0B9634B5D7A1A7A1F699D
:104410001543624EB6F86A309B0702D5202002F0A1
:10442000A7FF4FF000084FF0814AA37823B9BDE8F9
:10443000F88F857E876BECE794F80190B9F1000F57
:10444000F5D1D80715D5217811F0C00067D013F049
:10445000040B11D14146584684F80AB001F020FD02
:104460005846FDF747FAA37823F0020343F004030C
:10447000A370FFF70BFED8E7802912D10B2000F0C4
:104480007BFA0021484601F00BFD4846FDF732FA61
:1044900001F0C2FD63780BB1BDE8F88FFFF7F6FDC0
:1044A000F8E7402906D102F011FD18B9A37823F0EE
:1044B0002003A370A3781907DBD5DFF8DCB09BF8E5
:1044C00009204AB19A0707D4B6F86A309B071CD571
:1044D000237943F0080323719BF808305BB1A3787C
:1044E000980708D405F04000FDF704FA01214FF0C9
:1044F0007E50FFF7B7F8A3789907BAD443F01003BA
:104500000220A37002F08AFDB3E7394605F03000BF
:1045100001F0C6FC01215046FFF7A4F8DCE7A37ABE
:104520004BB39A0708D51C4B5B7AE3B1414601F0C7
:10453000B7FC0123A3729CE713F00C0F99D0164B24
:104540005B7A53B10A2000F017FAB6F86A3099077F
:104550000BD5237943F008032371A37A1A0702D5F8
:10456000022002F05BFD0023E4E7394605F030004D
:1045700001F096FCF1E723791B077FF57AAF394606
:1045800005F0300001F08CFC237923F0080323713F
:104590006FE700BF880D0020C80C002050100020DD
:1045A000454B2DE9F041B3F86A30444E13F0080F43
:1045B00007D0FEF743FA20B101230720337000F043
:1045C000DBF9337813F0810314D0022000F0D4F922
:1045D0000123337000242546394F00F09FFEFF2849
:1045E00017D1FFF749FDFFF705FF7378002BF4D0D3
:1045F000BDE8F081337002F069FC30B1314A1378C4
:1046000043F020031370FFF7F5FE2D4802F094FCF1
:10461000E0E70A2801D00D282BD1FFF7EBFE96F832
:104620000180B8F1000FE3D107F80480FEF716FC13
:1046300015F0010505D00B2000F076F9444625461B
:10464000CBE73C78002CFAD0242C06D1384602F077
:10465000EFFC00F069F92C46F1E7337813F0210400
:1046600001D00920F5E73846FDF722FA00F05CF9A1
:10467000E5E735B12928B0D1AB07AED505F0FD058A
:10468000ABE72028A9D92F28A7D028280DD03B2870
:104690000DD04E2C0DD8A0F16103DBB2192B98BFC1
:1046A0002038631C3855DCB297E7022595E70425CE
:1046B00093E7012591E700BF50100020880D0020EE
:1046C00004060020A50D002010B5FFF7D5FC064C10
:1046D000FFF790FE637833B9FFF75EF90028F7D152
:1046E0002378082BF4D010BD880D00200148FFF777
:1046F00095BB00BF5DA4000808B55D2000F0C4FDB7
:10470000BDE80840FFF7F2BF10B50446202000F0D6
:10471000BBFD282000F0B8FD212C52D8DFE804F0C2
:10472000111B1D1F21232527292B2D2F31335151DB
:104730005151513537393B3D3F4143454751494B35
:104740004D4F3648FFF76AFB292000F09DFDBDE87C
:104750001040FFF7CBBF3248F4E73248F2E7324867
:10476000F0E73248EEE73248ECE73248EAE7324811
:10477000E8E73248E6E73248E4E73248E2E7324821
:10478000E0E73248DEE73248DCE73248DAE7324831
:10479000D8E73248D6E73248D4E73248D2E7324841
:1047A000D0E73248CEE73248CCE73248CAE7324851
:1047B000C8E73248C6E73248C4E73248C2E7324861
:1047C000C0E70023A4F16400C0B20928DCB203F101
:1047D000010306D804280AD8DFE800F0060F1113F9
:1047E00015000A38C0B2F0E72848FFF717FB032C82
:1047F000AAD8DFE804F00A0C0E102548F5E7254892
:10480000F3E72548F1E72548EFE725489AE72548EB
:1048100098E7254896E7254894E700BFE9A40008F3
:10482000F3A40008FDA40008B2A5000805A500082F
:1048300010A5000818A5000820A5000831A500084B
:104840004BA5000863A5000867A500086FA5000830
:1048500077A5000880A5000898A50008A0A5000875
:10486000A8A50008AFA50008BAA50008C2A50008C1
:10487000CAA50008D3A50008DEA50008F4A5000815
:10488000FCA5000804A600080AA6000834A6000833
:10489000FBA4000810A6000812A6000814A6000831
:1048A00016A600081EA6000826A600082EA60008C8
:1048B0000148FFF7B3BA00BFE6A4000838B50546C3
:1048C000002455F82400FFF765FB042C02D02C20AF
:1048D00000F0DAFC0134052CF3D138BD10B50446E4
:1048E000242000F0D1FC2046FFF7A1FABDE81040DB
:1048F0003D2000F0C9BC10B50C46FFF7EFFFE0B259
:10490000FFF795FABDE81040FFF7F0BE38B50C464A
:104910001546FFF7E3FF29462046FFF7D7FABDE823
:104920003840FFF7E3BE000010B5044620B9BDE8EB
:1049300010400648FFF772BA0548FFF76FFA2046A5
:10494000FFF775FABDE81040FFF7D0BEDAA4000803
:10495000DFA4000810B504460648FFF75FFA2046BA
:10496000FFF765FAFFF7C2FEBDE810404FF4FA709A
:10497000FEF79ABEE8A2000810B504461448FFF7F7
:104980004DFA601E0A280AD8DFE800F0060D0F1164
:10499000131517191B1D1F000E48FFF73FFABDE83E
:1049A0001040FFF7A3BE0C48F7E70C48F5E70C48AA
:1049B000F3E70C48F1E70C48EFE70C48EDE70C484B
:1049C000EBE70C48E9E70C48E7E70C48E5E700BFF0
:1049D00046A300084CA300085EA3000872A30008C9
:1049E00084A300088CA3000895A30008A0A30008D6
:1049F000ADA30008B5A30008C8A30008DAA3000807
:104A000008B54FF4FA70FEF74FFEBDE808400148C4
:104A1000FFF704BA43A400080148FFF7FFB900BF3D
:104A2000F9A300082DE9F0477E4C002094F85010BF
:104A3000FFF761FF94F854100120FFF75CFF94F832
:104A400051100220FFF757FFB4F852100320FFF770
:104A500052FFB4F86A100420C1F38001FFF74BFF46
:104A6000B4F86A100520C1F38011FFF744FFB4F8D1
:104A70006A100620C1F3C011FFF73DFF94F8815082
:104A80000720FFF72BFF2846FFF7F9F9FFF72EFE67
:104A90000720FFF739FED4F884500820FFF71EFFE7
:104AA0002846FFF7ECF9FFF721FE0820FFF72CFE60
:104AB000D4F888500920FFF711FF2846FFF7DFF9E7
:104AC000FFF714FE0920FFF71FFE94F855100A2087
:104AD000FFF711FF0322A16D0B20FFF717FF032241
:104AE000E16D0C20FFF712FF94F86A100D2001F021
:104AF0000101FFF700FF94F868501320FFF7EEFE66
:104B00002846FFF7BCF9FFF7F1FD1320FFF7FCFD86
:104B1000B4F86A101420C1F34011FFF7ECFEB4F8AA
:104B20006A101520C1F3C001FFF7E5FEB4F86A1062
:104B30001620C1F30011FFF7DEFE94F86C10172069
:104B4000FFF7D9FE0322216F1820FFF7DFFE0322B3
:104B5000616F1920FFF7DAFEB4F878101A20FFF71A
:104B6000CAFE0322E16F1B20FFF7D0FE94F88000FD
:104B7000FCF784F8002201461C20FFF7C7FE1C202A
:104B8000FFF7C2FD0022216E1E20FFF7BFFE0022AC
:104B9000616E1F20FFF7BAFEB4F86A102020C1F33F
:104BA0004001FFF7A8FEB4F86A102120C1F30021EC
:104BB000FFF7A1FE4FF000086425DFF86CA02C463B
:104BC0006F1D184E5FFA88F9FFB2B9F1030F0BD8C9
:104BD000DFE809F002181B22032231682046FFF7A4
:104BE00095FE2046FFF790FD0134E4B2BC4206F189
:104BF0000406EAD10A35EDB2962D08F10108DED19E
:104C0000BDE8F08703227169E8E75146B06AFCF716
:104C100041F903220146E1E7F16B032201F1004172
:104C2000DCE700BF50100020000061457FB50B4855
:104C3000FFF7F4F80A4901A802F0B0F901A8FFF75C
:104C40003DFE3A2000F020FB064B5879FFF7EFF8C5
:104C5000FFF752FD07B05DF804FB00BF75A4000824
:104C6000A80D0020880D00202DE9F0410025234EDD
:104C7000234FDFF8A48086B0ECB201A9204600F0F3
:104C8000A2FD50B91F48FFF7C9F80720FFF7CFF87A
:104C9000FFF72CFD06B0BDE8F0813046FFF7BEF807
:104CA000062C07D0072C27D004F13600C0B2FFF73E
:104CB000BEF802E03846FFF7B1F83A2000F0E4FA17
:104CC000013501A8FFF7FAFDFFF716FD082DD3D136
:104CD0000D48FFF7A3F80D48FFF7F0FDFFF70CFDB7
:104CE0000B48FFF79BF80B4BD86DFFF753F9FFF715
:104CF00003FDFFF79BFFCDE74046DCE760A400081B
:104D000063A40008DFA4000869A40008100D0020B7
:104D10006FA40008C80C002066A4000810B5484C19
:104D20004848FFF77BF820788B2805D94648FFF7DD
:104D300075F820787630C0B2FFF779F84348FFF76E
:104D40006DF8A0793630C0B2FFF771F83F48FFF731
:104D500065F820791130C0B2FFF769F83B48FFF7DA
:104D60005DF8A078C0F11500C0B2FFF760F83748D1
:104D7000FFF754F8E0785A30C0B2FFF758F83348DC
:104D8000FFF74CF86078C0F15E00C0B2FFF74FF853
:104D9000E37973B1FFF78CFDE079032806D01E2874
:104DA00001D0022805D1FFF742F802E0302000F0E0
:104DB0006BFAFFF77DFD637A102B04D0202B38D0DF
:104DC00023B9352000E0332000F05EFAFFF770FDD4
:104DD000A37A23B1FFF76CFD362000F055FAFFF7F8
:104DE00067FD237A3BB31A0604D5FFF761FD372030
:104DF00000F04AFA237A5B0604D5FFF759FD382004
:104E000000F042FA1248FFF709F8207EFFF70FF88A
:104E10001048FFF703F86069FFF7D0F80E48FEF777
:104E2000FDFF20690021FFF751F8BDE81040FFF7B2
:104E300063BC3420C8E7FFF73BFD3920E0E700BF43
:104E4000C80C0020E3A30008E9A30008EDA30008B4
:104E5000F0A30008F3A30008F6A3000838B5054640
:104E60000C460848FEF7DAFF2846FEF7E0FF3D2033
:104E700000F00AFA2046FEF7D1FFBDE83840FFF700
:104E800035BC00BFD7A4000838B505460C463E2007
:104E900000F0FAF92846FEF7C1FF3A2000F0F4F9D5
:104EA0002046BDE83840FFF73FBD000010B504467E
:104EB0001C48FEF7B3FF2046FEF7B0FFFFF71CFCCF
:104EC0001948FEF7ABFF2046FEF7A8FFFFF714FCDA
:104ED0001648FEF7A3FF2046FEF7A0FFFFF70CFCE5
:104EE0001348FEF79BFF562000F0CEF94D2000F04E
:104EF000CBF95A2000F0C8F9482000F0C5F94C2041
:104F000000F0C2F92C2000F0BFF90F20FEF78FFF50
:104F10002C2000F0B9F9FE20FEF789FFBDE8104013
:104F2000FFF7EABBEFA2000803A3000824A30008D0
:104F300040A300082DE9F04FA94D91B001AC0FCD71
:104F40000FC42B680DF11809236001A94846A54C30
:104F500002F024F83C2000F097F92378082B4FD07A
:104F600031D8012B52D047D3022B51D0042B4BD038
:104F70009D4B93F85570984617F001075AD10025BC
:104F80009A4E0DF12C0BD6F85CA0303604367169C0
:104F90003068FBF7C3FD022D4BF8250003D15146C5
:104FA000FBF7BCFD0D903FB959F825005BF82510C3
:104FB000FBF7B2FD49F825000135052DE6D1002F9C
:104FC0003BD18B483AE0202B1CD00FD8102BCFD1EF
:104FD00094F90230002B15DB8648FEF71FFFA378FB
:104FE000DF0723D5302000F04FF9C1E7402B11D067
:104FF000802BBDD1804800E08048FEF70FFFB7E767
:105000007F48FAE77F48F8E77F48F6E77F48F4E70C
:105010007F48F2E77F48FEF701FFA3781E0701D51E
:105020003320E0E75D0703D59806DBD53120DAE7CA
:105030003220D8E7237B002BA1D07748FEF7EEFE85
:105040004846FFF73BFC98F8553099070ED5734852
:10505000FEF7E4FEFEF7C0FEFEF7E9FE2C2000F0AE
:1050600013F900F0E7F8C0B2FEF7E1FE6C48FEF776
:10507000D5FE01F0EDFDFEF7A1FF2C2000F004F9B4
:1050800000212069FEF722FFFDF7D8FC064601F05B
:1050900001FF0546FEF7C4FF46EA0503034313F08C
:1050A000FF0F07463AD05F48FEF7B8FE17B1502011
:1050B00000F0EAF8C6B1F20702D5582000F0E4F893
:1050C000B30702D5592000F0DFF8770702D55A2040
:1050D00000F0DAF8300702D5412000F0D5F8F106EB
:1050E00002D5422000F0D0F8C5B1EA0702D544202D
:1050F00000F0CAF8AB0702D5522000F0C5F86F07E0
:1051000002D5482000F0C0F82E0702D5532000F049
:10511000BBF8E80602D5462000F0B6F8237B6BB159
:10512000013B2373E37A23B3013BE3723E2000F09B
:10513000ABF8FFF7DBFA11B0BDE8F08F23789906E2
:1051400005D53948FEF76AFE0BA8FFF7B7FB2378B1
:1051500013F07C0F14BF1D2313232373E37A0BB9C1
:105160000123E3723048FEF759FE0BA8FFF7A6FBB8
:10517000D8E723782D4813F07C0F14BF13230E2398
:10518000E372FEF74BFEE079FEF751FE2C2000F0B3
:105190007BF8207AFEF74BFE2C2000F075F8607A41
:1051A000FEF745FE00F092FC0546FCF75DFB044669
:1051B0000DB90028BAD01E48FEF730FE2DB1012DE2
:1051C0000CBF5320432000F05FF8E20702D54620D1
:1051D00000F05AF8A307A9D54D2000F055F8A5E72F
:1051E000BC0D0020880D002050100020C80C0020AD
:1051F000B2A4000884A40008A5A400087BA40008A9
:1052000080A400088AA400088EA4000893A40008C3
:1052100099A400089FA40008ABA40008B9A4000842
:10522000BEA40008C3A40008C8A40008CEA40008B7
:10523000D3A40008064B074A1B8812889BB29342EE
:1052400094BF03F1FE0003F1FF30801A80B2704773
:10525000580600205606002007B501211020FCF753
:10526000A3F902238DF8063048238DF807304FF458
:10527000804302A921F8043D0248FCF76FF803B00F
:105280005DF804FB00100140F8B51C4E07464FF4D2
:1052900080411B483478FCF7BBF840B939461948BF
:1052A000FCF7D8FA174A13881906FCD5F8BD013463
:1052B000E4B2802C08BF0024134A14491378A34297
:1052C00017D03378124AD754124B1B78022B0ED1C9
:1052D000114D01222888394680B200F1005000F5B6
:1052E0009870FCF791FB2B8801339BB22B803470B4
:1052F00002E00B78DB06E1D5F8BD00BF5A060020BE
:1053000000100140003801405B060020A50D002080
:10531000D40D0020880D002054060020094A0A49B7
:10532000138809889BB2994209D0084911F81300E3
:1053300001339BB2FE2B08BF002313807047FF2070
:10534000704700BF5806002056060020540E00206B
:10535000F8B504464E4D4F4F4618B44200D1F8BD43
:1053600014F8013B212B54D046D8182B4AD01A06EA
:105370007DD5843B1D2BF0D801A252F823F000BF4D
:10538000175400081B5400085B5300085B530008C7
:105390005B5300085B5300085B5300085B53000835
:1053A0005B5300085B5300085B5300085B53000825
:1053B000275400082F5400083354000837540008BD
:1053C0003B5400083F540008435400084754000869
:1053D0005B5300084B54000853540008575400080E
:1053E0005B5400085F540008635400085B530008D6
:1053F000675400086B5400083F2B06D07E2BB6D1B3
:10540000022003E0FEF794F8A7E7012001F006FE72
:10541000A3E70820FAE72020F8E71F4B1B789B063C
:105420009BD54020F2E7012001F098FF95E702208C
:10543000FAE70420F8E70820F6E71020F4E7202038
:10544000F2E74020F0E78020EEE7012001F090FF36
:1054500083E70220FAE70420F8E70820F6E71020A7
:10546000F4E72020F2E74020F0E78020EEE72888EC
:105470003988421CD2B2FE2A08BF002289B292B2F9
:105480008A421EBF05492A8021F8103065E700BF17
:105490005606002058060020880D0020540E0020DB
:1054A00013B53D4A13889BB20193019B98062CD5F6
:1054B00093889BB2DAB2212A2DD017D8182A1BD094
:1054C000190656D5843A1D2A18D8DFE802F0262896
:1054D000171717171717171717172E323436383AAA
:1054E0003C3E17404446484A4C174E503F2A0ED087
:1054F0007E2AE5D102200BE0FEF71AF8264A13882F
:1055000023F020031B041B0C138002B010BD0120EC
:1055100001F084FDF2E70820FAE72020F8E71F4BAE
:105520001B789B06EAD54020F2E7012001F016FF28
:10553000E4E70220FAE70420F8E70820F6E7102065
:10554000F4E72020F2E74020F0E78020EEE701209A
:1055500001F00EFFD2E70220FAE70420F8E7082066
:10556000F6E71020F4E72020F2E74020F0E7802063
:10557000EEE70B480B4904880988631CDBB2FE2B5D
:1055800008BF002389B29BB28B421EBF064903802D
:1055900021F81420B2E700BF00380140880D002038
:1055A0005606002058060020540E0020024B1A8890
:1055B000024B1A80704700BF560600205806002094
:1055C00038B505460C46FFF77FF8512303FB05F07D
:1055D0002146BDE83840502200F54070FCF714BA6F
:1055E0000146502240F2AE30FCF70EBA38B50546FF
:1055F0000C46FFF769F8152303FB05F02146BDE8CB
:105600003840142200F50070FCF7FEB908B50A21F5
:105610000020FCF7F3F9BDE80840C422014901204D
:10562000FCF7F2B95010002030B50446E00787B00F
:1056300050D56421414B0A2283F85410C3F88410DA
:10564000C3F888101F2183F855103D4983F8502076
:1056500099653C490022D9653B4983F85120196678
:105660004FF07E515966032183F86C10374983F857
:1056700081201967364983F868205967FA2150223A
:10568000A3F8781033490120D9670421A3F86A20D0
:10569000314AA3F852001A605A609A602F4A83F880
:1056A0008010DA601A612E4A5A619A612D4ADA61D5
:1056B0001A625A622C4A9A62DA621A635A639A63CD
:1056C0002A4ADA632A4A1A642A4A5A649A64DA64C9
:1056D000FFF79CFFA1070CD51422002101A803F0BD
:1056E00084F80025E8B201A90135FFF77FFF082DF6
:1056F000F8D1620713D500214FF44070FCF77EF912
:10570000002140F20130FCF779F9002140F25130DC
:10571000FCF774F9002140F25230FCF76FF92307CF
:1057200009D5002140F2AE30FCF768F9002140F2C3
:10573000AF30FCF763F907B030BD00BF5010002058
:105740000AD7233C6F12033B00803B4600001644FF
:1057500000803B45000020400000A04200002043A4
:105760000080BB440000FA434054094B000066C36C
:105770000000A0C3000048C370B50D46512141434D
:105780000646502201F540712846FCF757F90446B9
:1057900030B9287029463046FFF712FF204670BD09
:1057A000012070BD38B5502240F2AE310546FCF7FD
:1057B00045F9044628B928702846FFF711FF20460E
:1057C00038BD012038BD70B50C4615214143064651
:1057D000142201F500712046FCF730F9054658B94E
:1057E0000023304623606360A360E36023612146A9
:1057F000FFF7FCFE284670BD012070BD08B50020F3
:10580000FCF7F6F80A2808D1C42201210448FCF765
:1058100015F9003018BF012008BD002008BD00BFE9
:105820005010002038B50C46054600212046FBF7F5
:105830001BFC002840F02D81632D34D9A5F16403B1
:10584000DBB2042BC2B225D8032A06D8DFE802F067
:1058500002090E1B934A42F82340FFF7D7FE0020AF
:1058600038BD904A02EB83035C61F6E78E4920461F
:1058700003F10A05FBF75AFA8B49FBF757FA894BF4
:1058800043F82500E9E7874A04F1004402EB83036B
:10589000DC63E2E7092B40F2FE800130052800F0CE
:1058A000FA800A3BCCE7204603F006F9FBF740FC00
:1058B000C0B2212D00F2EF80DFE815F022002900B0
:1058C0002D003300370043004D005C00600067008E
:1058D0006E00720075007800ED00ED00ED00ED0047
:1058E000ED0086008D009900A700B100B500B8005A
:1058F000BB00BF00C200ED00CC00D100D400DE0030
:10590000022840F2CA80674B83F85000A5E7654B38
:1059100083F85400A1E7634B83F8510000F02AFD9F
:105920009BE7604BA3F85200F8E75E4BB3F86A20A0
:1059300020B142F00402A3F86A208EE722F00402AC
:10594000F9E7584BB3F86A2010B142F04002F2E791
:1059500022F04002EFE7534BB3F86A2038B142F02F
:1059600080020020A3F86A20FEF73CFB75E722F0D6
:105970008002F6E74B4B83F881006EE72046FBF789
:10598000D7FB484BC3F8840067E72046FBF7D0FB02
:10599000444BC3F8880060E7424B83F855005CE74E
:1059A000404B9C6559E73F4BDC6556E73D4BB3F8F0
:1059B0006A2030B142F00102A3F86A2001F0D6FA61
:1059C0004BE722F00102F7E72046FBF7B1FB354B2E
:1059D00083F8680041E7334BB3F86A2020B1D10661
:1059E0005DD542F02002A6E722F02002A3E72D4B6E
:1059F000B3F86A2030B142F00802A3F86A20FDF73C
:105A000013F82AE722F00802F7E7264BB3F86A20DA
:105A100010B142F010028EE722F030028BE7214BEA
:105A200083F86C0019E71F4B1C6716E71D4B5C677A
:105A300013E71C4BA3F878000FE71A4BDC670CE761
:105A40002046FBF775FB174BC0B283F8800000F0CF
:105A500059F802E7134B1C6693F88000F7E7114BE7
:105A60005C66F9E70F4BB3F86A2010B142F480721C
:105A700061E722F002025EE70A4BB3F86A2028B120
:105A800042F48072A3F86A20122038BD22F480729A
:105A9000F8E7042038BD032038BD062038BD0A20B1
:105AA00038BD00BF501000200000704208B5FFF75D
:105AB000A5FE48B90720FEF737FFFF20FFF7B4FD2A
:105AC000BDE80840FEF7AEBF08BD000008B50448B9
:105AD000FBF7A4FC10F0040F14BF0220012008BD46
:105AE000000C014008B500210448FBF732FEBDE878
:105AF0000840012202210248FBF798BC0008004040
:105B0000000C014070B5022410258AB00646012120
:105B10000820FBF749FD694681488DF803508DF850
:105B20000240FBF71BFC69467D48ADF80040FBF7DF
:105B300015FC01217A48FBF780FC01210820FBF7C6
:105B400033FD8DF803500425694675488DF80240F1
:105B5000ADF80050FBF702FC21467148FBF76DFCE5
:105B6000002221466E48FBF761FC002229466C4862
:105B7000FBF75CFC01210920FBF716FD01212846FB
:105B8000FBF71EFD0DEB0500FBF73AFC1823012186
:105B900028468DF807308DF80640FBF711FD614A65
:105BA0006148D36900212B43D361FBF7C7FD5E48F1
:105BB000FBF7A7FD0F2E16D8DFE806F00874787CF7
:105BC00080848892969A9A9EA2A6AAAE4EF66022E9
:105BD000564B1B68B3FBF2F3013BADF80C3040F2BF
:105BE000E733ADF81030002403A94F48ADF80E405C
:105BF000ADF81240FBF7F0FC01210420FBF7E0FCBC
:105C000001214948FBF784FD02266023ADF81E40C0
:105C1000012406A94448ADF81830ADF81A40ADF893
:105C20002060FBF723FD08213F48FBF77DFD21465F
:105C30003D48FBF74FFD21460820FBF7B5FC02A8C5
:105C4000FBF7DEFB4FF40075182302A934488DF8EA
:105C50000B30ADF808508DF80A60FBF77FFB21464A
:105C60000420FBF7ADFC21462F48FBF733FD294606
:105C70002B48FBF7D9FBBDF81040601FFBF702F87B
:105C80002B4B0546596E186EFAF746FF014628461B
:105C9000FBF700F9274B1860274B1C80FFF722FF0A
:105CA0000AB070BD214B254A1B6893E71F4B244A5D
:105CB0001B688FE71D4B234A1B688BE71B4B224A4F
:105CC0001B6887E7194B214A1B6883E7174B204A5B
:105CD0001B68B3FBF2F3013BADF80C30632380E7A4
:105CE000124B1C4A1B6875E7104B1B4A1B68F0E7F8
:105CF0000E4B154A1B68ECE70C4B144A1B68E8E78F
:105D00000A4B164A1B68E4E7084B124A1B68E0E797
:105D1000064B134A1B68DCE7044B124A1B68D8E7A2
:105D2000000C014000100240000800401800002054
:105D300050100020141100201811002048E8010024
:105D400090D0030020A1070040420F0060E316003E
:105D5000E093040020AA4400C0270900C0C62D001B
:105D6000808D5B00E07072002DE970430646FAF703
:105D700041FB174C8046B4F840508946ADB22846E6
:105D8000FAF738FB0022134BFAF79AFB02460B4650
:105D900040464946FAF724FEB8B931462046BDE8E8
:105DA0007043FBF7D6BCB4F840102046013189B2ED
:105DB000FBF7CFFC95F86800FDF776FCB4F84030AF
:105DC0009BB29E42EFD8BDE87083034DF6E700BF5B
:105DD000000800400000F43F5010002010B50446B9
:105DE00001460948FBF7B5FC214607481CB9BDE848
:105DF0001040FBF7AEBCFBF7ACFCBDE81040002246
:105E000002210248FBF712BB00080040000C0140D1
:105E1000F8B51E4B05465E6E1F6E30463946FBF7E1
:105E200037F91B4C68B9607AFAF72CFF1949FAF771
:105E30007DFF2946FAF77AFF39460546FBF728F930
:105E400018B1154B27611888F8BD31462846FBF775
:105E500015F958B1002728463946FBF7FBF810B171
:105E600027610020F8BD26610520F8BD3146256177
:105E70002846FAF751FE094B1968FAF757FF02F066
:105E8000AFFDFBF755F9053080B2F8BD501000208A
:105E9000880D00200AD7233C18110020141100207F
:105EA00070B51B4C064662780D4632B930B90023F6
:105EB0002361FFF717FE0023E37270BD102818BF9F
:105EC000012204211348FBF7B1FA134BB3F86A20FF
:105ED000920702D5202E08BF002593F8683053B9E9
:105EE0002846FFF795FFFFF779FF002202210948B6
:105EF000FBF79CFADFE7094B094EB3F84030284620
:105F00003380FFF785FF3188FFF72EFFEDE700BFF5
:105F1000880D0020000C01405010002000080040B7
:105F2000C408002038B5074B04461B780D46022BE9
:105F300007D0FEF7C9FB29462046BDE83840FFF7E9
:105F4000AFBF38BD880D0020DFF834D0002103E05A
:105F50000C4B5B58435004310B480C4B42189A428F
:105F6000F6D30B4A02E0002342F8043B094B9A4265
:105F7000F9D301F017FA02F005FCFCF783FF704734
:105F80000050002030A9000800000020F801002087
:105F9000F801002094110020FEE7000038B5184CED
:105FA0004FF40041B4F86A20164812F0040218BFFA
:105FB0000122FBF73BFA144B144D1B681448AB61EC
:105FC00094F850300124043BC3EBC30203EBC2033B
:105FD000DB439BB2EB82013B9BB2838521468482EB
:105FE000FBF7BAFB4FF08042EB6B5B68013B9BB267
:105FF000938594824FF08052064B1A6038BD00BFE3
:106000005010002000100140B00800203807002088
:106010000004004000E100E04FF08052154B10B545
:10602000C3F880200022144C144B94F854001A70CA
:10603000FF28134B07D1134A117801F0FF0211B961
:106040001978802905D11B78042B11D0FDF72CFB82
:106050000122B4F86A305B0748BF82F0010202B146
:106060000122BDE810404FF400410748FBF7DEB9BC
:106070000022EEE700E100E0501000205C06002066
:10608000880D0020D00D0020001001402DE9F041C6
:106090004FF080473B8ADB0740F114813B8A914DEA
:1060A00023F001031B041B0C3B820023BB842B78D1
:1060B000002B40F007818C48FBF7B3F98B4E20F49E
:1060C000F070F169400421F4FC41400C21F01F0103
:1060D000014389B28448FBF7AEF901218448FBF7FC
:1060E0003BFB8148FBF79DF9B16920F01F0001439C
:1060F00089B27D48FBF79FF94FF000527D4BD6F8EF
:106100003C801A60012334462B70B8F1000F44D153
:10611000794A7A49138809889BB2994200F0D48061
:106120000C20138899B24843754B1E187268E663B9
:10613000013A92B2BA851A5894F83600A286327A99
:1061400090420DD01C266F4884F8362006FB0202D0
:10615000A263526952082261E260A260626022601A
:10616000A26B694E108B36687040E0610C2000FB1A
:1061700001331068597AC84020625068C840606294
:106180009068C840A062D0681269C840E06222FAF4
:1061900001F158892163FFF721FE5C4B1B78012B2D
:1061A00001D1FDF74DFF00232268A361A16B236A93
:1061B0001A444B6922609A420DD90120D21A2260FA
:1061C0000A8BA06112F0200F514A106814BF00F131
:1061D000FF30013010606268606A0244934262607E
:1061E0000FD2D21A62600A8BA06912F0400F484A9F
:1061F00040F00200A061506814BF00F1FF30013090
:106200005060A268A06A02449342A2600FD2D21AE0
:10621000A2600A8BA06912F0800F3D4A40F0040092
:10622000A061906814BF00F1FF3001309060E26817
:10623000E06A02449342E2600FD2D21AE2600A8B13
:10624000A06912F4807F324A40F00800A061D06853
:1062500014BF00F1FF300130D0602269206B02448E
:10626000934222610FD2D31A2361B1F91830A06989
:10627000002B274B40F010001A69A061B4BF02F157
:10628000FF3201321A61234B1A78042A01BF9A792E
:10629000A3691340A361A38E013B9BB2A38653B9AC
:1062A000154AE3631388013303F0FF030C2B08BF87
:1062B00000239BB21380184AA36912685340A3615C
:1062C00000232B70BDE8F081FFF7A6FEB36B9B7E29
:1062D00013B14046FFF782FDBDE8F041042000F015
:1062E0009DBE00BF5C06002000080140380700206A
:1062F0000004004000E100E03207002030070020E9
:10630000A00600207807002060060020A60D0020CF
:10631000BC0D0020880D0020B0080020114A08B5EF
:10632000138ADB071CD5138A0F4823F001031B04D3
:106330001B0C1382002393844FF000520B4BC3F8C5
:106340008020FBF76EF80A4B20F01F001968BDE8AB
:10635000084001F01F01014389B20348FBF76BB805
:1063600008BD00BF000400400008014000E100E05B
:10637000B008002000232DE9F04317481D4690F88F
:106380005170B0F852E01E4618461C461349144A94
:10639000DFF850C0DFF850800B60136047FA03F954
:1063A00019F0010F18BF5CF823604EFA03F91CBF07
:1063B0003443012619F0010F18BF58F8235003F198
:1063C00001031CBF28430125052BE7D106B10C6052
:1063D00005B11060BDE8F08350100020B008002027
:1063E0006006002060A6000838A6000838B5204CDA
:1063F000FFF712FE382200211E4802F0F6F9402273
:106400000021204602F0F1F9002301211A4A1B4D18
:1064100013601B4A13801B4A13801B4A11801B4ABE
:106420001370FFF7A7FF2B68E361194C2046FAF7BA
:10643000F8FF184B20F01F00196801F01F010143FD
:1064400089B22046FAF7F7FF2046FAF7EAFF2968F3
:1064500020F4F07021F4FC414004400C21F01F01B5
:10646000014389B22046BDE83840FAF7E4BF00BFD7
:10647000380700206806002064060020600600201F
:106480003207002030070020340700205C0600207F
:1064900000080140B008002038B5084C25685DB1FF
:1064A000074B5A78D96942F001025A700846FAF748
:1064B0003DFC0023E861236038BD00BF6406002076
:1064C000680600202DE9F04FA04B8DB01B79DC074A
:1064D00000F136814FF0000B9D4B9E4A1B881288BD
:1064E0009BB29A4200F02C819B4D2B68002B52D11D
:1064F000964B1B79580740F12681FDF741FA286039
:106500002F68002F00F01C81944C94F8018018F043
:10651000010100F02D8100236370D5F80090C4F8CC
:1065200018B0D9F824704FF07C503946FAF7B2FC15
:10653000864B80461B79D9F8286013F0020200F0E0
:1065400077810223D9F81C8023754146FAF7EEFBC8
:1065500001463046FAF7E0FA59468146FAF784FDDB
:10656000002800F0608139463846FAF7D7FA3146FC
:10657000FAF7DCFB01464046FAF7CEFAF9F74CFF92
:1065800002F0AEFAFAF774FA6062704B6F4A1B7948
:1065900043F008031371724B724A1B886F4C0093CF
:1065A0000C23009903FB0123227821691A722B68BE
:1065B00002939B6A18460693FAF7AEFA5946099079
:1065C000FAF752FD08B1CDF824B0A36AD4F820A0A0
:1065D0000393E36A03980793A36907990893636A8F
:1065E000E56994F814800A93FAF734FD002800F066
:1065F000D4814FF0020300275B4EDBB2DDF8189028
:106600000B930497CDF804B00596B8F1010F00F094
:106610001F82029B3046596AC0F0E481B8F1030F33
:1066200040F03382FAF782FB514607462846FAF7D4
:1066300073FA01463846FAF72BFD002800F0B281C4
:1066400003990698FAF768FA0146FAF767FA2946B5
:1066500004465046FAF762FA01462046FAF71AFC59
:10666000012706465546B846039C049731460198D3
:10667000FAF754FA019001460598FAF713FD00283D
:1066800000F0348201990598FAF746FA089906460F
:106690002046FAF707FD002840F08281049A2F4B2C
:1066A0000AB183F8148007B1DD61304B274E1B68B7
:1066B0002A4D9A7E12B93379180719D5029B9B7E11
:1066C00013F0300300F02082029B9F6B42B1296BD4
:1066D000E869FAF72BFB01463846FAF727FB07462D
:1066E0003846FFF795FBA886337923F0080333710A
:1066F0000C27009BDFF86C805F43A98E08EB070234
:1067000051812046E968FAF711FB029002F028F95E
:106710008146A86802F024F949468246FAF7FCF956
:10672000FAF706FD83B248F807304746002B40F0E1
:10673000EF813279910740F1EB8142F00102327131
:106740000DB0BDE8F08FFDF727F9D8E6880D0020E1
:10675000320700203407002064060020680600206D
:1067600030070020A00600205304E938AC080020C0
:1067700023781C260133DBB20B2B08BF0023944A7D
:106780009448964606FB03260660388B23703083B8
:1067900057F82120D20046F8212001310529F7D1F0
:1067A0001C2202FB03E37869C2005A61FAF766FA19
:1067B000B96AA060FAF76EFB0146E0608648FAF716
:1067C00069FB864B20611B79C4F804B0990702D499
:1067D00018F0080F1ED0616A28F00808E161084629
:1067E000FAF7A4FA84F80180F8610023B3767C4BB1
:1067F000B3F86A309A077FF590AEBB7E9B067FF5B3
:106800008CAE796B4FF07E50FAF744FB0123206386
:10681000B37682E6F869F9F7FFFD02F061F9FAF75D
:1068200027F9E061E1E7C4F81890C4F824B0ACE6B9
:10683000A6625E0722753FD5DA46C4F824B0286800
:10684000FDF7E0F801460290FAF770FA2B688146EE
:1068500000939B6A0193009BDE693146FAF704FCC2
:10686000002841D049463046FAF756F94146FAF732
:106870005DFA01460198FAF74FF95946A062FAF716
:10688000FDFB20B302232375009B596A0846FAF7E3
:1068900045F90199FAF74AFA01463046FAF73CF908
:1068A000F9F7BAFD02F01CF9FAF7E2F863786062D2
:1068B00043F00803637068E6FDF780F88246F9F755
:1068C000ABFD02F00DF9FAF7D3F86062B7E7514675
:1068D0004846FAF721F94146FAF728FA029BE062A6
:1068E00023620323237550E651463046FAF714F924
:1068F0004146FAF71BFA0199FAF710F94FF07C516B
:10690000FAF714FA59460746FAF7CCFB00283FD0AD
:1069100039460198FAF7C6FB002837D05146484659
:10692000FAF7FAF84146FAF701FA0146E06238460A
:10693000FAF7B8FBA8B1029B314623624846FAF742
:1069400089FB08B10123CDE731464846FAF7E4F860
:106950004146FAF7EBF90146A06AFAF7DDF8A062C2
:1069600013E6009BA762596AE7620846FAF7D6F871
:106970003946FAF7DBF95146FAF7D0F8F9F74CFD4A
:1069800002F0AEF8FAF774F82062FEE50223A9E7F8
:10699000636AC4F828B02362F7E54FF001032AE6E2
:1069A000A14632E64FF07C513846FAF7BFF901466E
:1069B0002846FAF7B1F83146FAF7B8F901464846E1
:1069C000FAF7AAF8044639462846FAF7A5F83CE053
:1069D00078070020AC0800200000A03F880D0020B0
:1069E00050100020FAF7A2F94FF07C510746FAF751
:1069F0009DF92946FAF792F83146FAF797F90146D8
:106A00004846FAF789F8044601460398FAF74AFB24
:106A1000B8B103990698FAF77FF80146FAF77EF8BD
:106A2000294604465046FAF779F801462046FAF717
:106A300031FA012706465546DDF82C80039C049761
:106A400014E639462846FAF769F8054601270DE6A7
:106A500051463046FAF76AF901464846FAF75CF8BB
:106A600007990446FAF700FB00283FF4FFAD0799A9
:106A70004846FAF751F85146FAF70CFACDF810806B
:106A80000646079C4FF00208F0E5FAF74FF9294651
:106A90000746FAF7E9FAA8B14FF07C513846FAF701
:106AA00045F901462846FAF737F83146FAF73EF934
:106AB00001464846FAF730F808990446FAF7F2FA20
:106AC000002880D108994846FAF726F80146FAF7D7
:106AD00025F8294604460A98FAF720F80146204688
:106AE000FAF7D8F90A9D0646089CAFE709992046AF
:106AF000FAF7D8FA00283FF4D1AD4E490598FAF7D5
:106B00000DF801990590BFE5C6F810B0AB86EBE52E
:106B1000019869680393FAF701F8029901905046C9
:106B2000F9F7FAFF019A01461046FAF7B3F9424A1B
:106B3000424912688246B2FBF1F048430192FAF7EB
:106B40009DF85146FAF7F2F83D49FAF7EFF801F0EF
:106B500007FFFAF7EDFA48F6A041019A039BB2FB52
:106B6000F1F188423AD20C23009A03FB027300220F
:106B70005A720C23009AB0F5803F03FB027728BFBE
:106B80004FF0FF332F4A28BF7B602F49138838BF4F
:106B900078600B8001339BB20C2B08BF00232B4F76
:106BA00013803B6802999C62C5F808904846F9F743
:106BB000B3FF5146FAF7BAF8A96968602046FAF7B8
:106BC00049FA00283FF488AC59462046FAF76AFA99
:106BD000337940B343F001033371B1E544F25061BE
:106BE000B2FBF1F1884210D20C22009902FB017233
:106BF000012151720C21009A51437A18527AD040E7
:106C000003FA02F248F80120B3E742F22831B2FB5E
:106C1000F1F290424FF00C02009902FB017234BF76
:106C200002210321E5E713F00402D3D13A60FCF717
:106C30008FFE51E45304E9381800002040420F0051
:106C40000000704234070020300700206406002056
:106C5000044B1B7813F07C0F1ABF034BD86900203C
:106C6000704700BF880D00206806002030B5013A4B
:106C700085B00446ADF8042000220139ADF80810B3
:106C800001A91D46ADF80A20ADF80620FAF7A4FCCC
:106C900001212046FAF760FD012220461146FAF74D
:106CA0002EFD01212046FAF715FD4FF44070FAF74A
:106CB0005FFAB4F1804F0ED11C238DF80030012310
:106CC00068468DF801508DF802308DF80330FAF7E0
:106CD00059FA05B030BD054B9C4201D11D23ECE7AC
:106CE000034B9C42EBD11E23E7E700BF00040040AA
:106CF000000800402DE9F3414FF400464FF0020830
:106D0000102702AC224D01211020FAF74DFC24F887
:106D1000046D214628468DF806808DF80770FAF735
:106D20001DFB01210420FAF73FFC48F2FF13214626
:106D30001848194CADF804308DF806808DF80770AE
:106D4000FAF70CFB314628460022FAF76FFBE3699D
:106D50004FF0804043F00103E36101231A461946D6
:106D6000FFF784FFE3690D4843EA0803E361012369
:106D70001A461946FFF77AFF4FF00052084BC3F846
:106D800080204FF08052C3F8802002B0BDE8F0812F
:106D900000100140000801400010024000040040C3
:106DA00000E100E070B5012186B00920FAF7FCFB94
:106DB00002238DF8063048238DF807304FF6E15353
:106DC00006A921F8143D3148FAF7C8FA0521012037
:106DD000FAF76CFB06210120FAF768FB2C4C07211F
:106DE0000120FAF763FB08210120FAF75FFBB4F8F2
:106DF0006A20120743D50A210120FAF757FB0C211C
:106E00000120FAF753FB0B210120FAF74FFB0D216C
:106E10000120FAF74BFB0E210120FAF747FB4FF652
:106E2000E053049300238DF81430102301250DEB5B
:106E300003008DF8153002268DF81650FAF7D0F9B8
:106E4000172302A88DF808308DF809608DF80A60C4
:106E50008DF80B50FAF796F9B4F86A301B0711D584
:106E600028238DF80C30032303A88DF80D608DF8CE
:106E70000E308DF80F50FAF785F906B070BD4FF45B
:106E8000F073CEE7FBF7D2FDF7E700BF000C01403F
:106E90005010002008B50C48FAF7C0FA88B180F409
:106EA0008073C3F30023820658BF43F002034106F8
:106EB00058BF43F00403020601D443F00803D8B2DC
:106EC00008BD0346FBE700BF000C014008B5FFF713
:106ED000E1FF00F0010008BD08B54FF4F070FAF7CB
:106EE000C7F9FFF7D7FF40B1830707D5FCF720FBB1
:106EF0004FF400020E4BC3F8802108BD010705D5F1
:106F00000C4A137843F002031370F1E7420704D5EB
:106F1000084A137843F00803F6E7C307E8D5FFF7FC
:106F2000D5FF0028E4D0034A137843F02003EBE7B1
:106F300000E100E0A50D002038B5044600252146FB
:106F4000E8B2FEF719FC40B9072120702046FDF792
:106F50009BFF0135022DF2D138BD2378002BF8D0EC
:106F60002046FAF7A5FD0146F0E7000008B5FDF759
:106F7000ABFB0022014B1A7308BD00BF880D002037
:106F800010B50C4650F82100F9F77CFE024B53F87F
:106F90002410F9F77FFF10BD5010002070B5054692
:106FA0000E460024A1B23046FFF7EAFF45F8240060
:106FB0000134052CF6D170BD2DE9F843804600253B
:106FC0004FF00009144C94F86C703C3447FA05F308
:106FD00058F8256013F0010F4946304611D0FAF7F2
:106FE00043F8B0B92168304601F10041FAF75AF888
:106FF00078B90135052D04F10404E7D10020BDE87E
:10700000F883FAF74FF820B921683046FAF72CF8E0
:10701000EEE70120BDE8F8835010002072B6034A65
:1070200013781843107062B6704700BFA50D00209A
:107030007FB5012344780546432C8DF8073003D0F3
:107040000BD884B1242C58D1AD78D5B9432C3CD081
:107050001DD8242C29D0002407E04A2C08D0582C15
:10706000F2D0472CEFE7FDF7D7FC204604B070BD07
:10707000A94B1B7813F0DF0F40F04B8183783D2B39
:1070800001D00324F1E7FAF713FD0446EDE7472C9E
:1070900014D0582CDFD1A04D2B78012BDBD1FFF77A
:1070A00015FF044620B30D24DFE79B4B1C7814F03A
:1070B000180440F02E81FDF7B5FCD6E7964B1B78FF
:1070C000002BC8D0FDF72AFEC5E7934B1C78022C95
:1070D00005D1FCF72DFA0520FDF74EFCBBE7002C8F
:1070E00040F01781022204201A70FDF745FCBCE72E
:1070F0000320FDF741FC2C70B7E7874E3378012B56
:1071000000F20781492C68D005D8232C1FD0482CC9
:1071100023D00024ACE0522C7DD0532C4DD04E2CEB
:10712000F7D10222AC788DF80720002C40F09D802A
:10713000E6B229463046FEF71FFB002840F090805B
:107140000720FDF7F1FB0134022C84D0F0E7AC7886
:10715000002C96D1FDF788FD87E7704BB3F86A30B5
:10716000DB0640F1D480FFF7B1FE00289BD1042359
:107170003370AB7883B9FCF74FF97478002C7FF447
:107180006AAF3470FEF748FFAB78002B7FF463AF33
:107190002846FFF7D1FE68E7EA78002A7FF471AF4E
:1071A000592B06D05A2B06D0582B7FF46AAF0120FA
:1071B000E1E70220DFE70420DDE7AB784C2B7FF42A
:1071C00060AFEB78502B7FF45CAF2C79002C7FF410
:1071D00058AF8020FFF722FF47E70223AC788DF8F5
:1071E000073034B92846FEF7DDFA2846FDF75EFE83
:1071F0003BE73D2C7FF445AF0323EC5CEA180133F9
:1072000002F8034CDBB2002CF7D128468DF807308A
:10721000FEF7E6F929E7AB78532B7FF432AFEB7832
:10722000542B7FF42EAF2B793D2B7FF42AAFAB7913
:10723000002B7FF426AF6B79242B06D02A2B0DD0A0
:10724000232B7FF41EAF022000E00120FEF7ECF9B3
:107250000920FDF791FBFCF76BF9FCE6FF20F5E751
:1072600029463046FDF7FAFD6DE7002B51D1012488
:1072700002AA0DF107012846FCF784F908B9022497
:10728000F3E69DF807305A1CEB5CD2B23D2B8DF82B
:1072900007207FF4F6AEE4B11346EC5C981AE918C7
:1072A0002C5409780133DBB20029F6D128468DF839
:1072B0000730FAF7FDFB044600287FF4D6AE0298AB
:1072C00001F0FAFBF9F734FF2946C0B2FEF778F96E
:1072D000CBE603AA0DF107012846FCF753F9002875
:1072E000CDD09DF80730EB5C002B7FF4CAAE029C3A
:1072F0000B492046F9F7D6FE00287FF4C2AE20469F
:10730000F9F716FF0399C0B2FEF78CFABDE6052423
:10731000ABE60824A9E600BF880D0020501000202D
:1073200000007F4372B6034A137823EA000010700E
:1073300062B67047A50D002072B6034A1378184351
:10734000107062B6704700BFD00D002072B60022E8
:10735000014B1A7062B67047D00D002072B6034A16
:1073600013781843107062B6704700BF850D002077
:1073700072B6034A13781843107062B6704700BFA4
:10738000A40D002072B60022014B1A7062B670473D
:10739000850D002072B60022014B1A7062B670474C
:1073A000A40D0020374B82B01A6842F001021A6027
:1073B0005968354A0A405A601A6822F0847222F4E9
:1073C00080321A601A6822F480221A605A6822F405
:1073D000FE025A604FF41F029A600022009201924E
:1073E0001A6842F480321A601A6802F4003201927C
:1073F000009A01320092019A1AB9009AB2F5A06F70
:10740000F2D11A6812F4003218BF01220192019AD7
:10741000012A05D04FF000621C4B9A6002B0704701
:107420001B4A116841F010011160116821F003013D
:107430001160116841F0020111605A685A605A687F
:107440005A605A6842F480625A605A6822F47C1288
:107450005A605A6842F4E8125A601A6842F0807220
:107460001A601A689201FCD55A6822F003025A6029
:107470005A6842F002025A605A6802F00C02082A66
:10748000FAD1C7E7001002400000FFF800ED00E06D
:107490000020024010B5074C002220464FF4005156
:1074A000F9F7C4FF2046BDE8104000224FF48041A8
:1074B000F9F7BCBF000801402DE9F3414FF4005635
:1074C0004FF002081027174C02AD01210420FAF7F3
:1074D0006BF825F8046D294620468DF807708DF865
:1074E0000680F9F73BFF01210420FAF75DF88DF8DB
:1074F00007704FF48047294620468DF80680ADF886
:107500000470F9F72BFF394620460022F9F78EFF69
:10751000002231462046F9F789FFFFF7BBFF02B092
:10752000BDE8F0810008014000224FF400510148FD
:10753000F9F77CBF0008014000224FF48041014868
:10754000F9F774BF0008014038B50F4C657825B9CC
:1075500020B9FFF7E9FF0023E37238BD0228FAD112
:107560000A4B18700A4B0B48D3F884306361F9F763
:1075700058FF83044CBF2A4601224FF400510548AE
:10758000F9F754FFE7E700BF880D0020840D0020C5
:10759000501000200008014038B50C4C65782DB91A
:1075A000012804D1FFF7C8FF0023E37238BD042887
:1075B000FAD10748F9F735FF43044CBF2A460122A8
:1075C0004FF480410248F9F731FFEDE7880D0020C4
:1075D0000008014010B5064B04461B78022B06D06C
:1075E000FDF772F82046BDE81040FFF7D5BF10BD8B
:1075F000880D002010B5064B04461B78022B06D0E0
:10760000FDF762F82046BDE81040FFF79DBF10BDB2
:10761000880D002010B5064C18B9012223681A8283
:1076200010BD044B1B681B68984720680A3010BDCA
:10763000481100204411002010B5064C18B9012251
:1076400023681A8210BD044B1B689B68984720680A
:107650000C3010BD481100204411002010B5204B03
:1076600018B902221B681A8210BD00201D491C682F
:10767000088023780A4613F07F0313D1637A9906B2
:1076800044BF0221117013F0400F137814BF43F070
:10769000010323F001031370134B1B681B69984708
:1076A000104810BD012B18D0022B17D1617901F0C1
:1076B0000F039B0003F1804303F5B84311F0800FE3
:1076C0001B6805D003F03003102BE5D10123E2E75E
:1076D00003F44053B3F5805FF7E7084610BD00BFE1
:1076E000481100201A110020441100202DE9F84310
:1076F000234FDFF8A0803D682C8AD4B92E7A042E5F
:1077000017D120490B68012B0ED11F4B1A681F4B54
:1077100092B213445B001C6030230C60A8F8003068
:107720003B681E72BDE8F88310230726A8F80030D6
:10773000F6E7AB8A9C4294BF042602269C4228BFEF
:107740001C46AB69204698478146002000F076FD34
:1077500022460146484600F047FC2146002000F042
:107760000DFD2B8A4FF440521B1B2B826B8A1C444D
:107770003023A8F80030064B6C821A80D0E700BF97
:1077800048110020B4080020505C00400230002066
:107790004E1100205011002010B50A4B0A491B68F9
:1077A0004978DA7891420AD3997841B99C8834B9FA
:1077B0009A72064B1B685B689847204610BD0220F2
:1077C00010BD00BF48110020B0000020441100206F
:1077D00038B50F4A0F4D12682B689269D9785879DD
:1077E00090472B6804469A7A7AB170B91A7962B9CF
:1077F0009B7853B9084B1B68DB6898472B685A790C
:10780000DA72DA781A73204638BD0224FBE700BF2B
:1078100020110020481100204411002038B5304BC1
:107820001B68187810F07F0004D15A7A22F02002E9
:107830005A7238BD022850D15A88002A4ED11A797E
:10784000002A4BD15979274D21F08000840004F1A2
:10785000804202F5B842126849B22D780029B4BFBF
:1078600002F0300202F44052A84236D2002A34D04C
:107870009B7A93B304F1804404F5B844002923684B
:1078800011DA03F03003102B07D1C4B2204600F008
:1078900062FC3021204600F0E1FB134B1B685B6962
:1078A0009847002038BD03F44053B3F5805FF4D10E
:1078B0000E4D78B90E4B93F82C1000F06DFC236838
:1078C0002B409BB283F4405343F4004343F08003C6
:1078D0002360E2E700F02CFCF1E7022038BD00BF96
:1078E00048110020B0000020441100208FBFFFFF8E
:1078F0008000002038B51F4B1F4D18682D78417946
:1079000021F08004A30003F1804202F5B84212681E
:1079100049B20029B4BF02F0300202F44052AC4236
:1079200025D244881CBB12B3827A02B303F1804390
:1079300003F5B8431A680029B5BF22F4E04222F4E7
:10794000804222F0400222F07002B5BF92B292B2A1
:1079500082F0100282F4805242F4004242F080022F
:107960001A60064B1B689B699847002038BD0220AF
:1079700038BD00BF48110020B00000204411002095
:1079800008B5064B1A68537A43F020035372044B30
:107990001B68DB699847002008BD00BF4811002024
:1079A00044110020054B10B51C68628A18B98B88F9
:1079B0009B1A238210BD0868104410BD4811002096
:1079C00008B50B4B002093F82C1000F0E5FB094B99
:1079D0001B68187A082806D14FF48052064B1A808B
:1079E0001022064B1A80A0F109035842584108BDE5
:1079F00080000020481100204E110020501100206E
:107A0000F7B5984C984E276832683B7A092B19D005
:107A1000964B92B213445B001D886D0005F18045C2
:107A200005F5C0452B783B706B787B70A88800F01B
:107A300029FC78802889276800F024FCB880AA896E
:107A40002368DA80012223681A72DA885D78002AB6
:107A500063D11A7812F07F024CD1092D03D1FFF7C0
:107A60009BFEB0B126E0052D1FD193F90320002A1B
:107A700006DA082322681372FFF7A2FF03B0F0BDF5
:107A80009A78002AF5D19A88002AF2D19B7A002BA5
:107A9000EFD13268764B92B2134400225B001A6039
:107AA0003022744B1A800623E4E7032D14D1DA78D0
:107AB000012A08D0704B28461B685B699847032849
:107AC00028D10923D6E79A88002AF3D15B7A980651
:107AD000F0D5FFF755FFC4E7012DEBD1DA78012A85
:107AE000E8D19A88002AE5D15B7A9906E2D5FFF7BA
:107AF00095FEB6E7012A04D10B2DDBD1FFF768FE16
:107B0000AFE7022AD6D1012DF1D0032DD2D1FFF754
:107B1000F1FEA6E70028ACD1BBE7062D14D11A78F8
:107B200052065DD19A78544B012A03D11B68DB6958
:107B3000EBB955E0022A02D11B681B6AF8E7032A59
:107B40004ED11B685B6AF3E7002D55D15988002997
:107B500046D15A6822F47F42B2F5003F40D11A78EC
:107B600012F07F0216D19B88002B39D1434B0025A0
:107B70002268284655829361984728464FF6FF7140
:107B800023681A8A8A4234D0022801D0002A56D1AA
:107B900008222FE0012A0AD1374A587912689269DF
:107BA0009047E8B923689B7A002BDFD118E0022ABE
:107BB00016D15A79324802F00F018B0003F180434D
:107BC00003F5B8431B68007812F0800F14BF03F070
:107BD000300303F44053814202D212F0700FE3D01D
:107BE000254B22681B6850781B6998470328C5D12C
:107BF000236809221A723FE7082D04D11B785B061F
:107C0000EED1204BB3E70A2DEAD11A7802F07F02B9
:107C1000012AE5D19A7A002AE2D059880029DFD1D9
:107C20005A6822F47F42B2F5803FD9D1124A58797E
:107C30001268926990470028D2D1134B97E793F9C5
:107C40000010002935DAD9880B4C01910198824245
:107C50001CD9019A1A82226892F82C209A82FFF786
:107C600045FD09E748110020505C00400430002029
:107C70000230002050110020201100205D76000805
:107C8000B000002015760008397600088A42E2D25A
:107C9000216891F82C00824203D20021084A116029
:107CA000D9E792FBF0F100FB1122002AD3D1012188
:107CB000F4E703221A724FF44052024B1A80DBE6BB
:107CC000B40800204E110020F8B52C4D2C68237A02
:107CD000022B50D0042B4ED0032B01D0052B44D1C6
:107CE000A369268AABB1A6B1A28A964228BF1646DE
:107CF00030469847238A07469B1B2382638A0020CD
:107D00003344638200F0AAFA32460146384600F056
:107D10007DF9238A53B100214FF44052184B084695
:107D20001A8000F02BFA3022164B1A80A38A228A7E
:107D300093422B6809D803221A722B681B7A2A688F
:107D40001372BDE8F840FFF73BBE0AB10522F3E726
:107D5000062119720C4B19680C4B89B20B445B005D
:107D60001A603022074B1A80E7E7072B03D1084B34
:107D70001B68DB6898470823E1E700BF4811002033
:107D80004E11002050110020505C004002300020B5
:107D900020110020F0B5002240F60F7548F2800651
:107DA0000A4B1C78A24204D3094B40F080001860B3
:107DB000F0BD02F1805303F5B8539B00196842EA05
:107DC00006072940394319600132EBE7B000002073
:107DD0004C5C004010B5134C23681A7A022A01D07B
:107DE000042A09D1FFF782FC23681B7A22681372E8
:107DF000BDE81040FFF7E4BD062A10D15A78052AE5
:107E000009D11A78520606D1D878FFF7C3FF064B7E
:107E10001B681B6A9847054B1B689B68984708239B
:107E2000E4E700BF48110020441100202011002089
:107E300070470000064B074A0749136002221A7276
:107E4000064B074A1360074A1B681160184700BFBA
:107E50002811002048110020D400002080000020BC
:107E6000201100204411002000232DE9F743DFF802
:107E70007091DFF87081ADF80630D9F80030524AC1
:107E800099B21B0411804CD5138803F00F0388F8B6
:107E90000030002B65D14BF6BF764C4C4C4D23681F
:107EA0004C4F9BB22B802B8803F030033B802B88F8
:107EB00003F440532B802368334083F4005383F052
:107EC000200343F4004343F080032360138813F03E
:107ED000100F236828D123F4E14323F070031B041F
:107EE0001B0C2360FFF776FF23682A883340D604F3
:107EF0002A8848BF83F4805395043A8848BF83F4A6
:107F00000053D4063A8848BF83F01003900648BF58
:107F100083F0200343F4004343F080032B4A9BB2D9
:107F2000136003B0BDE8F0839BB2ADF80630BDF836
:107F300006301A0508D5236823F070031B051B0DB6
:107F40002360FFF75DFDCFE7BDF806301B0494D535
:107F5000236823F070031B051B0D2360FFF7B4FE9D
:107F6000C2E79A0002F1804202F5B842116889B274
:107F7000ADF80610BDF8061009040AD51168013BDA
:107F800021F070010905090D1160134A52F82330E0
:107F90009847BDF806301A067FF56FAF98F80020B5
:107FA000930003F1804303F5B8431968013A21F4C3
:107FB000E14121F070010904090C1960074B53F8E5
:107FC0002230984759E700BF92110020005C004022
:107FD0004E110020501100205400002038000020D5
:107FE000445C004024110020002310B501F1005131
:107FF000013201F54051521049009A4200D110BDA2
:1080000030F8024B21F823400133F6E7002310B586
:1080100001F10051013201F54051521049009A42DC
:1080200000D110BD51F8234020F813400133F6E78A
:108030004FF6F873014A034013607047505C0040EC
:10804000800000F1804000F5B840036823F4EC4361
:1080500023F07003194389B201607047800000F17A
:10806000804000F5B8400368CA0623F4E04323F0DB
:1080700040039BB248BF83F010038A0648BF83F0D9
:10808000200343F4004343F0800303607047800003
:1080900000F1804000F5B8400368CA0423F480432F
:1080A00023F070039BB248BF83F480538A0448BF17
:1080B00083F4005343F4004343F0800303607047AC
:1080C000800000F1804000F5B840036823F4E043ED
:1080D00023F040039BB283F0300343F4004343F0AA
:1080E000800303607047800000F1804000F5B840D5
:1080F000036823F4804323F070039BB283F440535E
:1081000043F4004343F0800303607047800000F1B4
:10811000804000F5B840036823F4F8731B051B0D7D
:1081200043F4004343F0800303607047FFF7EEBF62
:10813000800000F1804000F5B84003685B0409D579
:10814000036823F0F0031B051B0D43F4404343F089
:10815000800303607047800000F1804000F5B84064
:1081600003685B0609D5036823F0F0031B051B0DAC
:1081700043F4004343F0C00303607047044B1B68A3
:108180009BB203EBC000034B03445B0019607047D4
:10819000505C0040023000200D4B0E4A1B683E2907
:1081A0009BB203EBC00002444FEA42020AD94B09DA
:1081B000C80604BF03F1FF339BB29B0243F40043A4
:1081C000136070474B08C90748BF01339B02F7E7AC
:1081D000505C004006300020064B49081B684900EF
:1081E0009BB203EBC00000F1005000F5405040008E
:1081F00001607047505C0040FFF7EEBF054B490837
:108200001B6849009BB203EBC000034B03445B00B7
:1082100019607047505C004004300020FFF7EEBF4B
:10822000054B1B689BB203EBC00000F1005000F54A
:108230004050400000887047505C0040FFF7F0BF9E
:10824000044B1B689BB203EBC000034B03445B0071
:1082500018887047505C004004300020FFF7F0BFE2
:10826000054B1B689BB203EBC000044B03445B004F
:108270001868C0F309007047505C004006300020C9
:10828000FFF7EEBFC3B2000A40EA032070470000C8
:108290000020044B044A18604FF406431380034A3D
:1082A00013607047445C00404C110020405C00406B
:1082B00070B500F07F0528460E46FFF7E1FF044643
:1082C0002846FFF7CBFF224601463046FFF79EFEC9
:1082D000204670BD002330B51D46DCB2A24200D856
:1082E00030BD040F092C94BF3034373401F81340EB
:1082F00001EB4304000165700133EEE708B500208F
:10830000F9F708F9BDE8084001214FF40000F9F73A
:1083100057B937B54FF4C060F8F72AFF012414238A
:10832000002501A88DF804308DF805408DF8065021
:108330008DF80740F8F726FF2A2301A88DF80430AE
:108340008DF805408DF806508DF80740F8F71AFFB4
:1083500003B030BD70470000094B10B518685C6869
:1083600008331B68C0180AD008220649FFF7B2FF7D
:108370002046BDE8104004220349FFF7ABBF10BD03
:10838000E8F7FF1F1E0000202E00002010B5074C4C
:1083900003202146FFF78CFFC1B22046FCF7D8FF2F
:1083A000BDE810400320FFF79EBE00BF5211002021
:1083B000F8B5254B254D1B782A78934242D0244AA4
:1083C000126802F03002202A3CD12A7893428DBFF5
:1083D0002C782A7803F180041C1B98BFA41AA4B23D
:1083E00084B3402C1B4A28BF402417462B78611CBD
:1083F00019481344491013F8016B0430A3EB020E23
:10840000BEF1800F08BF3B4613F801EB46EA0E268B
:1084100020F8086C9E1A802E08BF3B460139EAD12D
:1084200021460120FFF7AAFE0120FFF749FE2B7825
:108430001C44E4B22C702B781B0642BF2B7883F0CF
:1084400080032B70F8BD00BF5A0600205B06002099
:10845000045C0040D40D002084610040034B1B6885
:10846000052B01D1FFF7A4BF704700BFC008002053
:108470007047000070B5164C164E2268164D92B229
:108480003280298832880A40910509D54FF6FF537A
:10849000124A236013780133DBB21370FFF7DEFF5B
:1084A0002A88338813401A0401D5FFF7DDFC33888E
:1084B0002A8813405B0509D54FF6FF332360084B2C
:1084C0005B689847BDE87040FFF7D2BF70BD00BF42
:1084D000445C0040921100204C110020B80800209C
:1084E00080000020034B9B7A13B10522024B1A60D7
:1084F000704700BF28110020C00800200422014B53
:108500001A607047C0080020034B1A78202A04BF65
:1085100000221A70704700BFB908002070470000A1
:10852000212810B50BD1134B1B681B7803F07F0378
:10853000212B1CD00022104B02201A6010BD2028D5
:10854000F8D10C4B0D4A1B681B78107003F07F03A9
:10855000212B0B4B18BF0023002BEBD00024054A26
:1085600020461268936154829847204610BD054BFF
:10857000F4E700BF48110020BC080020B908002023
:10858000C9850008E1850008094B1A68137803F0D3
:108590007F03212B0AD1022806D0222806D1D378C6
:1085A000044A03F001031360002070470220704763
:1085B00048110020BC08002021B901288CBF0220EE
:1085C000002070470220704720B90822024B1B6828
:1085D0001A8270470148704748110020F8000020B7
:1085E000FFF7F2BF10B50024FFF7B6FE044B1B687F
:1085F0009C7200F0A5F8FFF74BFE024B1C6010BD0B
:1086000048110020C008002010B50024324B334A26
:108610001B68D2799C725A72DC722046FFF708FD03
:108620004FF400712046FFF70BFD10212046FFF7A5
:1086300015FD40212046FFF7F1FD80212046FFF780
:10864000DBFD2046FFF772FD254B204693F82C10EA
:10865000FFF7A2FD2046FFF746FD21460120FFF768
:10866000EFFCC0210120FFF7C7FD20210120FFF70B
:10867000F5FC21460120FFF70AFD4FF4C0610220FE
:10868000FFF7DEFC4FF480710220FFF7B5FD2146B5
:108690000220FFF7FCFC20210220FFF7DFFC21462F
:1086A0000320FFF7CDFC4FF488710320FFF7B6FDE0
:1086B00040210320FFF770FD4FF440510320FFF7E6
:1086C000E6FC21460320FFF7C9FC2046FFF762FBCA
:1086D0000122044B1A6010BD4811002074A6000846
:1086E00080000020C00800200149FFF75BB900BFEF
:1086F000780000200149FFF755B900BF7000002045
:10870000054B1B68DB78042B04D8044901EBC3013B
:10871000FFF748B90020704748110020B40000203E
:10872000054B1B68052B05D1044B1868003018BF9A
:108730000120704700207047C0080020BC080020BE
:1087400008B50120FFF706FE01220020054B06496F
:108750001A60064A186010604FF4E0520A801A60EE
:1087600008BD00BF405C00404C110020445C00404C
:108770007047FEE7FEE7FEE7FEE770477047704789
:10878000FFF778BE70B500250C4E0D4CA41BA4104D
:10879000A54209D101F09CFD00250A4E0A4CA41BFC
:1087A000A410A54205D170BD56F825309847013573
:1087B000EEE756F8253098470135F2E728A900087A
:1087C00028A9000828A900082CA9000810B501391B
:1087D0000244904201D1002010BD10F8013B11F875
:1087E000014FA342F5D0181B10BD0346024493422B
:1087F00000D1704703F8011BF9E7000030B5184AB3
:1088000021F00043934287B004DC0022002300F0F3
:10881000D7FD06E0134A934205DD02460B46F7F703
:108820009BFC07B030BD02AA00F0D6FADDE90423B4
:1088300000F00304012CDDE9020108D0022C0CD069
:10884000002CE4D00124009401F0EEF9E9E7009453
:1088500001F0EAF901F10041E3E700F0B1FDF9E7C9
:10886000FB21E93FFFFFEF7FF8B50D46002DC5F373
:108870000A53A3F2FF36B4BF4FF0FF340124C5F30F
:108880001305132E45F480150FDC002E04DA013693
:1088900018BF00242046F8BD4FF4002333412B4479
:1088A000C6F11406F3405C43F4E71E2E1AD8332EAB
:1088B000A3F2134106DDA3F233438D4000FA03F324
:1088C0002B43F0E74FF00042CA401218C6F13403C0
:1088D00028BF0135202B05FA01F514BF22FA03F356
:1088E0000023EDE7F8F79CF80446D3E730B51A4AC1
:1088F00021F00043934287B006DC0023002200935E
:10890000002301F091F906E0144A934205DD024686
:108910000B46F7F721FC07B030BD02AA00F05CFA65
:10892000DDE9042300F00304012CDDE9020105D098
:10893000022C06D064B901240094E2E700F040FD67
:10894000E9E70124009401F06FF901F10041E2E749
:1089500000F036FDF9E700BFFB21E93FFFFFEF7FA5
:1089600070B520F00046F50D7F3D162D01460446FA
:1089700026DC002D0EDA1849F8F7D0F80021F8F7B8
:1089800091FB28B1002C23DB002E18BF4FF07E5442
:1089900021461BE0114E2E41304217D00E49F8F708
:1089A000BDF80021F8F77EFB0028F1D0002CC2BFF3
:1089B0004FF4000343FA05F5641924EA0604E7E7D7
:1089C000B6F1FF4F02D3F8F7A9F80146084670BD8B
:1089D0004FF00044DCE700BFCAF24971FFFF7F009F
:1089E00070B520F00046F50D7F3D162D014604467A
:1089F00026DC002D0EDA1749F8F790F80021F8F779
:108A000051FB28B1002C23DA134B002E18BF1C4653
:108A100021461BE0114E2E41304217D00D49F8F788
:108A20007DF80021F8F73EFB0028F1D0002CBEBFF6
:108A30004FF4000343FA05F5641924EA0604E7E756
:108A4000B6F1FF4F02D3F8F769F80146084670BD4A
:108A50000024DDE7CAF24971000080BFFFFF7F00FC
:108A6000C0F3C7530028A3F17F0210B5B4BF4FF085
:108A7000FF3401241E2A1BDC002A04DA013218BF4D
:108A80000024204610BD162AD8BF4FF48003C0F33F
:108A90001601D8BF134141F40001CDBF963B5B18CE
:108AA000C2F1170201FA03F3D8BFD3405C43E8E7F1
:108AB000F8F718FB0446E4E7C0F3C7537F3B162BD7
:108AC000024608DC002B02DA00F000407047024842
:108AD000184122EA00007047FFFF7F0000F0A0B8B5
:108AE0002DE9F04F8BB004460D4600F069FB244B96
:108AF000804693F900A08946BAF1FF3F2BD0224669
:108B00002B4620462946F7F775FF834618BB0026FB
:108B1000002732463B4620462946F7F743FFD0B1AF
:108B200001230093174BCDF820B00193CDE9044504
:108B3000CDE90245BAF1000F12D1CDE906676846CA
:108B400001F046FBB8B1089B1BB101F0BBFB089BD1
:108B50000360DDE90689404649460BB0BDE8F08F69
:108B600032463B4630463946F7F7D4FDBAF1020F9C
:108B7000CDE90601E3D101F0A5FB21230360E2E783
:108B800000010020FFA60008F0B58BB0044600F0FD
:108B9000C3FB204B064693F900506B1C2AD021469C
:108BA0002046F8F789FA074620BB00212046F8F74F
:108BB0005BFAF8B101230093174B20460193089705
:108BC000F7F72AFC0022CDE90401CDE902010023D8
:108BD0009DB9CDE90623684601F0FAFAA8B1089BD1
:108BE0001BB101F06FFB089B0360DDE90601F7F79D
:108BF0003FFF064630460BB0F0BD10461946F7F76A
:108C000089FD022DCDE90601E5D101F05BFB2123B1
:108C10000360E4E70001002004A700080000000052
:108C20002DE9F84F564223F0004E1643DFF8A0918D
:108C30004EEAD6764E4504460D46884607D846424B
:108C400021F00047064347EAD6764E4506D920462E
:108C50002946F7F783FA04460D4615E003F140462E
:108C600006F58016164303D1BDE8F84F01F094B81D
:108C70009E1706F0020646EAD17650EA070107D1B0
:108C8000022E30D0032E32D020462946BDE8F88F80
:108C900052EA0E0106D1B8F1000F71DA3AA5D5E912
:108CA0000045F1E7CE4526D1774511D1022E07D0F8
:108CB000032E09D0012E5DD135A5D5E90045E3E7A6
:108CC00035A5D5E90045DFE735A5D5E90045DBE762
:108CD000022E08D0032E0AD0012E4FF000044DD1F1
:108CE0004FF00045D0E730A5D5E90045CCE730A5E9
:108CF000D5E90045C8E74F45CDD0A7EB0E073F1596
:108D00003C2F1EDC002B01DA3C371EDB20462946B7
:108D1000F7F700FD01F0D2F901F03EF804460D46E8
:108D2000012E15D0022E16D0002EADD022A3D3E9ED
:108D3000002320462946F7F70FFA1BA3D3E90023A7
:108D400015E01FA5D5E90045EAE700240025E7E77F
:108D500005F1004598E718A3D3E9002320462946EA
:108D6000F7F7FAF902460B460FA1D1E90001F7F730
:108D7000F3F970E714A5D5E9004585E7002583E7F9
:108D80000FA5D5E900457FE7182D4454FB21F9BF15
:108D9000182D4454FB21E9BFD221337F7CD90240F6
:108DA000D221337F7CD902C0182D4454FB210940C5
:108DB000182D4454FB2109C0075C143326A6A13C9E
:108DC000182D4454FB21F93F182D4454FB21E93F51
:108DD0000000F07F000000002DE9F04F1446C44A67
:108DE00021F0004A92458DB08B4607DC002200231B
:108DF000C4E90001C4E90223002523E0BD4A9245ED
:108E000071DCADA3D3E900230029BB4D36DDF7F7B4
:108E1000A3F9AA4506460F4618D0A9A3D3E9002313
:108E2000F7F79AF902460B463046C4E90023394663
:108E3000F7F792F9A2A3D3E90023F7F78DF90125FB
:108E4000C4E9020128460DB0BDE8F08F9EA3D3E926
:108E50000023F7F781F99EA3D3E9002306460F46C6
:108E6000F7F77AF902460B463046C4E90023394643
:108E7000F7F772F996A3D3E90023DEE7F7F76EF967
:108E8000AA4506460F4616D08DA3D3E90023F7F76F
:108E900065F902460B463046C4E900233946F7F728
:108EA0005BF987A3D3E90023F7F758F94FF0FF35B3
:108EB000C4E90201C6E784A3D3E90023F7F74EF91A
:108EC00083A3D3E9002306460F46F7F747F9024686
:108ED0000B463046C4E900233946F7F73DF97CA339
:108EE000D3E90023E0E7854A924500F3D68001F0FC
:108EF000E5F879A3D3E9002306460F46F7F7E0FA31
:108F000000227F4BF7F72AF9F7F78AFD0546F7F7B6
:108F100071FA69A3D3E90023CDE90201F7F7D0FA8A
:108F200002460B4630463946F7F716F964A3D3E9F3
:108F3000002306460F46DDE90201F7F7C1FA1F2DAF
:108F4000804689462EDC6F4B6A1E53F822309A45C4
:108F500028D042464B4630463946F7F7FDF8C4E97B
:108F600000012368D4F804A00293029A53463046C5
:108F70003946F7F7F1F842464B46F7F7EDF8024667
:108F80000B46BBF1000FC4E90223BFF65BAF029BA7
:108F900001F1004123600AF100436360A060E160D9
:108FA0006D424FE742464B4630463946F7F7D4F814
:108FB0000B4602464FEA2A5AC1F30A51AAEB0101B5
:108FC0001029C4E90023CCDD3FA3D3E90023DDE968
:108FD0000201F7F775FA8046894602460B4630468D
:108FE0003946F7F7B9F8CDE9040102460B46304699
:108FF0003946F7F7B1F842464B46F7F7ADF834A3D8
:10900000D3E9002306460F46DDE90201F7F758FAD7
:1090100032463B46F7F7A0F802460B4680468946A3
:10902000DDE90401F7F798F80B460246C1F30A514F
:10903000AAEB010ABAF1310FC4E900232ADD28A303
:10904000D3E90023DDE90201F7F73AFA80468946C1
:1090500002460B46DDE90401F7F77EF802460B46AF
:1090600006460F46DDE90401F7F776F842464B461F
:10907000F7F772F81CA3D3E9002380468946DDE99F
:109080000201F7F71DFA42464B46F7F765F88046AE
:1090900089465EE7DDE9046763E71B4A924535DDF3
:1090A00002460B46F7F758F8C4E90201C4E900018B
:1090B000A2E600BFAFF3008000004054FB21F93F5F
:1090C0003163621A61B4D03D0000601A61B4D03DD2
:1090D0007370032E8A19A33B83C8C96D305FE43FC8
:1090E0000000002E8A19A33BC14920259A837B39B1
:1090F000FB21E93F7BD90240FB21F93FFB213941AC
:109100000000E03F0CA70008FFFFEF7F4FEA2A5561
:10911000A5F21645AAEB05510F460646F7F780FC67
:10912000F7F768F902460B4630463946CDE9062383
:10913000F7F712F80022204BF7F7C2F90F46064660
:10914000F7F76EFCF7F756F902460B4630463946FC
:10915000CDE90823F7F700F80022174BF7F7B0F92D
:109160004FF0030800260027CDE90A010DF1300970
:10917000324679E902013B4608F1FF3AF7F708FC6D
:10918000B8B90E4B2A46019302232146009306A844
:10919000434600F0F3F9BBF1000F0546BFF652AEAF
:1091A000636803F100436360E36803F10043E36035
:1091B000F6E6D046DCE700BF000070418CA700084F
:1091C0002DE9F041DFF84CE106463EEA010E0D467E
:1091D00007460A460C4603460FD102460B46F7F7F0
:1091E0006FF902460B4630462946F6F7B7FF0646AA
:1091F0000D4630462946BDE8F08100290EDC21F0FD
:10920000004E5EEA0707F4D041B102460B46F6F77E
:10921000A3FF02460B46F7F77DFAE8E712150CD1DB
:10922000002C6ED00021E6026FD5481E121AC1F143
:10923000200023FA00F004438B40A2F2FF32D5074E
:109240004FF00005C4F3130444F4801442BF6400DB
:1092500004EBD3745B0004EBD3715010214416224D
:109260002C464FF400165B00A7198F42DEBFC91BC6
:10927000BC19AD194900013A01EBD3714FEA56060A
:109280004FEA4303F0D14FF0200E94464FF00046D2
:10929000A14206EB0C0702DC12D19F4210D8002F2E
:1092A00007EB060C34DABCF1000F31DB04F10108E6
:1092B000091B44469F4288BF01F1FF31DB1B32444A
:1092C00001EBD377BEF1010E39444FEA43034FEA75
:1092D0005606DDD10B4306D0541C0BBF724601323B
:1092E000013522F001026B105208E90703F17F53A8
:1092F00003F5001348BF42F0004203EB0055164649
:1093000077E7DC0A153A5B058AE7640001318AE7F2
:10931000A046CDE70000F07F20F00042B2F1FF4F01
:1093200070B50346044609D30146F7F7FFFC014632
:109330002046F7F7F3FB0446204670BD002AFBD019
:10934000002806DA0146F7F7E7FB0146F7F7A2FD2A
:10935000F1E7B2F5000F4FEAE05404D200221902FF
:1093600029D5013AA41A7F3CE2074FF000024FEAE8
:10937000640116464FF019044FF08070C3F31603D2
:1093800043F4000348BF5B005B0035189D42DEBF1D
:109390002E185B1B1218013C4FEA43034FEA5000A2
:1093A000F3D113B1013222F00102541004F17C54C4
:1093B00004EBC154C0E75B000132D0E700000000BD
:1093C0002DE9F04F21F00047B7F1795F85B00546F0
:1093D0000C4692469B4604DAF7F722FB002800F081
:1093E000A8802A46234628462146F7F769F852A363
:1093F000D3E9002380468946F7F762F850A3D3E902
:109400000023F6F7ABFE42464B46F7F759F84EA35A
:10941000D3E90023F6F7A0FE42464B46F7F750F893
:109420004BA3D3E90023F6F799FE42464B46F7F7E4
:1094300047F849A3D3E90023F6F78EFE42464B4690
:10944000F7F73EF846A3D3E90023F6F787FE4B462D
:109450004246F7F735F8444BCDE900019F422ADC3C
:109460000022424B40464946F7F72AF8DDE900233F
:1094700006460F4640464946F7F722F852468046D0
:1094800089465B4628462146F7F71AF802460B46FE
:1094900040464946F6F760FE02460B4630463946DE
:1094A000F6F75AFE024600200B463149F6F754FE05
:1094B00005B0BDE8F08F2F4B00209F42DFBF002298
:1094C000A7F5001316461F46C4BF00262A4F324692
:1094D0003B462749F6F740FE0022CDE90201234B27
:1094E00040464946F6F7ECFF32463B46F6F734FE77
:1094F000DDE9002306460F4640464946F6F7E0FF01
:109500005246804689465B4628462146F6F7D8FFF4
:1095100002460B4640464946F6F71EFE02460B46FB
:1095200030463946F6F718FE02460B46DDE90201E1
:10953000BCE700200E49BBE7D43888BEE9FAA8BDD5
:10954000C4B1B4BD9EEE213EAD529C804F7E923E92
:109550009015CB19A001FA3E7751C1166CC1563F48
:109560004C5555555555A53F3233D33F0000E03F8C
:109570000000F03F0000E93F0000D23F2DE9F04F2E
:10958000ADF51B7D06930191C04BA499D41E53F8F1
:10959000213000250293069B0A90013B0893182373
:1095A00094FBF3F46FF0170324EAE47404FB033331
:1095B00003EB020A089A029BA71A03EB0208A59B79
:1095C000002203EB8709002320AE454514DD002669
:1095D0000DF5E07B029B9E4239DC0A9B4FF00008B0
:1095E000083B0493069B4FF000099D1922AB03EB47
:1095F000C5030993002723E0EF420BD459F8250057
:10960000CDE90423F6F7F6FEDDE90423E6E90201DD
:109610000135DAE710461946F8E70999049D71E922
:1096200002230991F5E902010495F6F749FF024684
:109630000B4640464946F6F791FD8046894601377C
:10964000089B9F42E9DDEBE902890136C2E7029BF4
:109650000EAA02EB83030D93A59B029F03EB8403E9
:109660000C9300269AAB07F1005B03EBC7030BF1E9
:10967000FF3B53E928894FEACB030993099A9AAB38
:109680001344A3F1980BBB1B002B70DC52464046E1
:10969000494600F0A1FD00224FF07F5304460D46DD
:1096A000F6F70EFF00F010FD0022794BF6F708FFE9
:1096B00002460B4620462946F6F74EFD0D46044667
:1096C000F7F7AEF90490F6F795FE02460B462046F2
:1096D0002946F6F741FDBAF1000F804689466BDD59
:1096E0007A1E0EAB53F82200CAF11801049C40FA0E
:1096F00001F31C448B40C01A0EAB43F82200CAF1A0
:109700001703049440FA03FBBBF1000F62DD002253
:109710006FF07F411446049B01330493974200F39A
:109720008880BAF1000F07DDBAF1010F00F09580D3
:10973000BAF1020F00F09B80BBF1020F4AD1424602
:109740004B4600205349F6F707FD80468946002C1A
:1097500040D0524600204F4900F03EFD02460B46E5
:1097600040464946F6F7F8FC8046894632E000223A
:10977000494B40464946F6F7A3FEF7F751F9F6F78D
:1097800039FE0022454B04460D46F6F799FE024687
:109790000B4640464946F6F7DFFCF7F741F90EABBA
:1097A00043F8260029467BE902232046F6F7D6FC3B
:1097B00001368046894666E706D17B1E0EAA52F81E
:1097C00023004FEAE05B9FE70022354BF7F7FEF8F6
:1097D00060BB83460022002340464946F7F7D8F88D
:1097E000002800F0C4807C1E2346002202998B4290
:1097F00044DA002A40F0888001246FF0030202FB63
:1098000004F30D99CB58002B3ED0099B9AAA134420
:10981000A3F1980B069B7E1CDD1902EBC505A5F58F
:10982000F4753C44A6423DDD27461AE74FF0020B93
:109830006DE70EAB53F822304CB92BB1C3F18073F6
:109840000EA840F82230012301321C4666E7CB1AED
:109850000EA840F822302346F6E77A1E0EAB53F8E6
:109860002230C3F316030EA941F8223064E77A1EB2
:109870000EAB53F82230C3F31503F4E70EA951F8E9
:109880002310013B0A43B1E70134B8E7D8A8000828
:10989000000020400000F03F0000703E00007041DA
:1098A0000000E03F05F108030B930C9B002753F8E1
:1098B0002600F6F79FFD4FF000084FF000090A9BC5
:1098C000C5E90201083B049305F110030993089BC5
:1098D0009F4204DDEBE9028901360B9DA2E709995D
:1098E000049D71E902230991F5E902010495F6F757
:1098F000E7FD02460B4640464946F6F72FFC013786
:1099000080468946E3E7013C0EAB53F82430AAF1C8
:10991000180A002BF7D052460020B54900F05CFC35
:10992000254606460F464FF00009E3009AAA02EBCF
:109930000308DFF8C4A20893A8F19808002D4CDAB8
:10994000002504F100580DF5907A08F1FF38631BEB
:10995000002B71DB72ABA8EB050703EBC7070022F6
:109960000023DFF89892CDE90623002659E0CAF1DA
:1099700000024046494600F02FFC00229D4B044661
:109980000D46F7F723F8F8B100229B4B20462946F5
:10999000F6F796FDF7F744F80646F6F72BFD00229A
:1099A000944BF6F78DFD0B46024629462046F6F706
:1099B000D3FBF7F735F87C1C0EAB43F827000AF110
:1099C000180A43F82460A6E720462946F7F728F846
:1099D0000EAB43F827003C469DE70EAB53F825003D
:1099E000F6F708FD32463B46F6F76AFD4A4668E957
:1099F0000201534630463946F6F762FD013D064600
:109A00000F469BE7F7E90223F9E90201F6F758FD53
:109A100002460B46DDE90601F6F7A0FBCDE906019B
:109A20000136029B9E4201DCAE42EBDDDDE90623FE
:109A30000135EAE902238AE7A49B032B6CD8DFE80F
:109A400003F0582C2C02089A4AAB9D18AA462646C9
:109A5000002E00F38880A246BAF1010F00F3A18026
:109A600000273E46089D4AAB08351D44012C00F3F3
:109A7000B580BBF1000F40F0C38001994AABD3E938
:109A80000023C1E900234CABD3E90023C1E9022341
:109A90003A463346C1E904233EE04FF0000E264625
:109AA0007746089D4AAB08351D44002E45DABBF1C8
:109AB000000F4CD007F1004172460B460199012678
:109AC000C1E900234AA97246D1E900013B46F6F7F5
:109AD00043FB86460F464AADB4423ADABBF1000F6B
:109AE00001D007F1004772463B460199C1E90223C4
:109AF00012E000273D46089B9AAA1344A3F59C76E2
:109B0000002C10DABBF1000F01D005F100453A46F8
:109B10002B460199C1E90023049B03F007000DF5D2
:109B20001B7DBDE8F08F384676E902232946F6F71B
:109B300015FB013C07460D46E2E7704675E9022336
:109B40003946F6F70BFB013E86460F46ADE7394630
:109B5000B2E77046F5E902233946F6F7FFFA013617
:109B600086460F46B8E7DAE900235AE902894046FB
:109B70004946CDE90223F6F7F1FACDE9060102469E
:109B80000B4640464946F6F7E7FADDE90223F6F7C9
:109B9000E5FADDE90623CAE90001013E6AE902238C
:109BA00056E7D5E9002355E9026730463946CDE945
:109BB0000223F6F7D3FA02460B4680468946304622
:109BC0003946F6F7C9FADDE90223F6F7C7FA0AF1D2
:109BD000FF3AC5E9000165E902893DE7384675E9C4
:109BE00002233146F6F7BAFA013C07460E463DE736
:109BF0000000F03F000070410000703E90A8000897
:109C0000019A4A9B06F1004613604B9B176103F1D2
:109C1000004353604C9B566193604D9B03F100439E
:109C2000D36079E7000000002DE9F04786B0CDE968
:109C3000002321F00043B3F1795F82460C460E9D6C
:109C400003DAF6F7EDFE002850D052462346504680
:109C50002146F6F735FC06460F4602460B465046AF
:109C60002146F6F72DFC3EA3D3E900238046894622
:109C700030463946F6F724FC3BA3D3E90023F6F738
:109C80006BFA32463B46F6F71BFC39A3D3E90023B7
:109C9000F6F764FA32463B46F6F712FC36A3D3E9F0
:109CA0000023F6F759FA32463B46F6F709FC34A38F
:109CB000D3E90023F6F752FACDE90201DDB90246F5
:109CC0000B4630463946F6F7FBFB2FA3D3E90023BA
:109CD000F6F742FA42464B46F6F7F2FB02460B46CF
:109CE00050462146F6F73AFA82460C46504621463F
:109CF00006B0BDE8F0870022DDE90001244BF6F74D
:109D0000DFFBDDE90223CDE9040140464946F6F7D1
:109D1000D7FB02460B46DDE90401F6F71DFA324691
:109D20003B46F6F7CDFBDDE90023F6F715FA16A35F
:109D3000D3E9002306460F4640464946F6F7C0FBE6
:109D400002460B4630463946F6F708FA02460B46FD
:109D500050462146F6F700FAC6E700BFAFF3008091
:109D60007CD5CF5A3AD9E53DEB9C2B8AE6E55A3EA5
:109D70007DFEB157E31DC73ED561C119A0012A3F41
:109D8000A6F810111111813F495555555555C53F3C
:109D90000000E03F000000002DE9F84FBA4B21F031
:109DA00000469E4204460D468B4617DDB74A964252
:109DB00001DC09D140B122462B4620462946F6F760
:109DC000CDF904460D4605E0BBF1000FB04C00F3A1
:109DD0002981B04D20462946BDE8F88FAE4B9E4202
:109DE00011DCA3F1DE739E420ADC8FA3D3E90023CA
:109DF000F6F7B4F90022A94BF6F7F2FD0028E9D1F5
:109E00004FF0FF3A27E000F059F9A54B04469E4277
:109E10000D4600F3B880A3F550239E4200F39C80CA
:109E200002460B46F6F79AF900229C4BF6F794F996
:109E3000002206460F464FF0804320462946F6F79B
:109E40008DF902460B4630463946F6F763FC4FF073
:109E5000000A04460D4622462B4620462946F6F7C0
:109E60002FFB02460B4680468946F6F729FB70A376
:109E7000D3E9002306460F46F6F722FB6EA3D3E98B
:109E80000023F6F76BF932463B46F6F719FB6CA355
:109E9000D3E90023F6F762F932463B46F6F710FBAA
:109EA00069A3D3E90023F6F759F932463B46F6F7A2
:109EB00007FB67A3D3E90023F6F750F932463B4688
:109EC000F6F7FEFA64A3D3E90023F6F747F9424612
:109ED0004B46F6F7F5FA62A3D3E90023804689469C
:109EE00030463946F6F7ECFA5FA3D3E90023F6F7DC
:109EF00033F932463B46F6F7E3FA5DA3D3E9002394
:109F0000F6F72AF932463B46F6F7DAFA5AA3D3E9CE
:109F10000023F6F721F932463B46F6F7D1FA58A36B
:109F2000D3E90023F6F718F932463B46F6F7C8FAAC
:109F3000BAF1FF3F02460B464ED140464946F6F77E
:109F40000DF922462B46F6F7BBFA02460B46204691
:109F50002946F6F701F934E70022504BF6F7FCF8F2
:109F6000002206460F464D4B20462946F6F7F6F8E6
:109F700002460B4630463946F6F7CCFB4FF0010A55
:109F800004460D4667E7474B9E421ADC0022464BCB
:109F9000F6F7E2F8002206460F46434B20462946D4
:109FA000F6F78EFA00223D4BF6F7D8F802460B463C
:109FB00030463946F6F7AEFB4FF0020A04460D462E
:109FC00049E702460B4600203849F6F7A3FB4FF05D
:109FD000030A04460D463EE740464946F6F7BEF8FA
:109FE00022462B46F6F76CFA314E324B4FEACA0A3C
:109FF00056449A44DAE90023F6F7AEF822462B4697
:10A00000F6F7AAF802460B46D6E90001F6F7A4F8DF
:10A01000BBF1000F04460D46BFF6DCAE01F1004374
:10A020001D46D7E6244DD5E69C7500883CE4377E76
:10A0300011DA22E33AAD903FEB0D76244B7BA93F3A
:10A04000513DD0A0660DB13F6E204CC5CD45B73F08
:10A05000FF8300922449C23F0D5555555555D53FB4
:10A060002F6C6A2C44B4A2BF9AFDDE522DDEAD3FA8
:10A070006D9A74AFF2B0B33F711623FEC671BC3F48
:10A08000C4EB98999999C93FFFFF0F440000F07FF6
:10A09000182D4454FB21F9BFFFFFDB3F0000F03FC8
:10A0A000FFFFF23FFF7F03400000F83F0000F0BFDA
:10A0B000E8A8000808A90008FB21F93F21F00041A9
:10A0C00070470000000000002DE9F843C1F30A5872
:10A0D000A8F2FF36132E07460B460C46054635DC24
:10A0E000002E16DA36A3D3E90023F6F737F800225C
:10A0F0000023F6F775FC48B1002C5CDA24F000432D
:10A100003B43314B4FF0000518BF1C4623462F46FA
:10A1100027E02E4A42FA06F801EA0802024320D05C
:10A1200027A3D3E90023F6F719F800220023F6F756
:10A1300057FC0028EAD0002CBEBF4FF4801343FA2E
:10A1400006F6A41924EA08040025DFE7332E0CDD07
:10A15000B6F5806F05D10B460246F5F7FFFF0746BF
:10A160000B4638461946BDE8F8834FF0FF32A8F297
:10A17000134822FA08F810EA080FF2D010A3D3E926
:10A180000023F5F7EBFF00220023F6F729FC002857
:10A19000BCD0002C02DA142E03D1013425EA0805C4
:10A1A000B4E70123C6F1340603FA06F63544AF429C
:10A1B00088BFE418F2E700252C46A7E7AFF300803C
:10A1C0009C7500883CE4377E0000F0BFFFFF0F0065
:10A1D0000020704700000000F8B51646C1F30A528F
:10A1E00004460D460B468AB921F00043034335D09F
:10A1F00000222D4BF6F764F92C4A044696420D4690
:10A200000B460EDA24A3D3E900231CE040F2FF77CB
:10A21000BA4209D102460B46F5F7A0FF04460D46A7
:10A220001CE0C1F30A52363A40F2FE7132448A42CF
:10A230000CDD22462B461AA1D1E9000100F03AF8C4
:10A2400017A3D3E90023F6F73BF9E7E7002A08DD77
:10A2500023F0FF4323F4E00343EA02552046294656
:10A26000F8BD12F1350F0BDA4CF250339E42224604
:10A270002B46E0DC08A1D1E9000100F01BF8C1E7A2
:10A2800023F0FF43363223F4E00343EA025520462D
:10A2900029460022064BD6E759F3F8C21F6EA501E6
:10A2A0009C7500883CE4377E00005043B03CFFFFC3
:10A2B0000000903C21F0004203F0004342EA030119
:10A2C00070470000014B1868704700BF0401002070
:10A2D000F8B500BFF8BC08BC9E467047F8B500BF93
:08A2E000F8BC08BC9E46704763
:10A2E800414C41524D3A005B5645523A312E316647
:10A2F8002E32303139303332333A005B4F454D3AE4
:10A30800417765736F6D652E74656368202E2053E1
:10A318007570657247657262696C3A005B534552A5
:10A328003A307830303030312E446174653A32300A
:10A338003139303133303A005B4F50543A005B4D7D
:10A3480053473A00526573657420746F20636F6ECB
:10A3580074696E756500272448277C2724582720B0
:10A36800746F20756E6C6F636B0043617574696FF1
:10A378006E3A20556E6C6F636B656400456E616262
:10A388006C65640044697361626C65640043686568
:10A39800636B20446F6F7200436865636B204C6980
:10A3A8006D6974730050676D20456E640052657363
:10A3B800746F72696E672064656661756C7473008A
:10A3C800526573746F72696E67207370696E646C1E
:10A3D8006500536C656570696E67005B47433A4773
:10A3E8000033382E00204700205400204600205318
:10A3F800005B484C503A242420242320244720245E
:10A408004920244E2024783D76616C20244E783DE6
:10A418006C696E6520244A3D6C696E652024534C36
:10A4280050202443202458202448207E2021203FE7
:10A43800206374726C2D785D0D0A000D0A477262F4
:10A448006C20312E3166205B27242720666F72200E
:10A4580068656C705D0D0A005B4700323800333068
:10A46800005B4739323A005B544C4F3A005B50521C
:10A47800423A0049646C650052756E00486F6C641E
:10A488003A004A6F6700486F6D6500416C61726DF4
:10A4980000436865636B00446F6F723A00536C65E4
:10A4A8006570007C4D506F733A007C57506F733A5B
:10A4B800007C42663A007C46533A007C506E3A0073
:10A4C8007C57434F3A007C4F763A007C413A00244F
:10A4D8004E006F6B0D0A006572726F723A00204D64
:10A4E800007374702070756C73650069646C206407
:10A4F800656C61790073747020696E76007374708E
:10A5080020656E20696E76006C696D20696E760034
:10A5180070726220696E7600415443204D362C20BB
:10A5280070756C73652F66660041544320546F6FD5
:10A538006C2054642C206D696C6C697365636F6E54
:10A54800647300415443204D362054642C206D69B7
:10A558006C6C697365636F6E647300727074006A03
:10A568006E63206465760061726320746F6C00729C
:10A57800707420696E636800536F667473746172D7
:10A58800742C206D696C6C697365636F6E647300FD
:10A59800736674206C696D00687264206C696D0064
:10A5A800686D2063796300686D2064697220696E44
:10A5B8007600686D206665656400686D2073656562
:10A5C8006B00686D2064656C617900686D2070753A
:10A5D8006C6C6F6666005370696E646C6520667299
:10A5E80065712E203020746F2031350072706D2017
:10A5F8006D61780072706D206D696E006C617365B5
:10A6080072006661756C74007A00610062003A73CA
:10A6180074702F6D6D003A6D6D2F6D696E003A6D17
:10A628006D2F735E32003A6D6D206D617800000009
:10A638002000000040000000800000000001000031
:10A648000080000000040000001000000008000066
:10A65800002000000040000001000000020000008F
:10A668000400000008000000100000000902430078
:10A67800020100C0320904000001020201000524A1
:10A68800001001052401000104240202052406002B
:10A6980001070582030800FF09040100020A0000FF
:10A6A8000007050302400000070581024000001270
:10A6B8000100020200004083044057000201020327
:10A6C80001040309041C03530054004D00330032F5
:10A6D8000046003100300033004300380054003693
:10A6E80000160374006F006D0065006B006F00209A
:10A6F800006E006500740073717274007371727477
:10A7080066000000FB21F93FFB2109407CD912407B
:10A71800FB2119407A6A1F407CD92240BBFD2540A5
:10A72800FB2129403A462C407A6A2F405C47314049
:10A738007CD932409C6B3440BBFD3540DB8F3740C1
:10A74800FB2139401BB43A403A463C405AD83D4078
:10A758007A6A3F404C7E40405C4741406C10424022
:10A768007CD942408CA243409C6B4440AC34454069
:10A77800BBFD4540CBC64640DB8F4740EB584840C1
:10A78800FB21494083F9A200444E6E00FC291500C4
:10A79800D1572700DD34F50062DBC0003C999500F5
:10A7A800419043006351FE00BBDEAB00B761C500BA
:10A7B8003A6E2400D24D42004906E00009EA2E0014
:10A7C8001C92D100EB1DFE0029B11C00E83EA70039
:10A7D800F535820044BB2E009CE98400B426700045
:10A7E800417E5F00D6913900538339009CF43900CB
:10A7F8008B5F840028F9BD00F81F3B00DEFF97003F
:10A808000F980500112FEF000A5A8B006D1F6D007D
:10A81800CF7E360009CB2700464FB7009E663F0023
:10A828002DEA5F00BA277500E5EBC7003D7BF10014
:10A83800F739070092528A00FB6BEA001FB15F00EC
:10A84800085D8D00300356007BFC4600F0AB6B00C2
:10A8580020BCCF0036F49A00E3A91D005E61910088
:10A86800081BE60085996500A0145F008D4068000C
:10A8780080D8FF0027734D0006063100CA56150020
:10A88800C9A873007BE260006B8CC0000000000068
:10A8980000000040FB21F93F000000002D44743EF9
:10A8A800000000809846F83C0000006051CC783BDE
:10A8B80000000080831BF0390000004020257A3812
:10A8C800000000802282E336000000001DF3693595
:10A8D8000200000003000000040000000600000061
:10A8E8004FBB610567ACDD3F182D4454FB21E93FA0
:10A8F8009BF681D20B73EF3F182D4454FB21F93F8F
:10A90800E2652F227F2B7A3C075C143326A6813C14
:10A91800BDCBF07A8807703C075C143326A6913CBF
:04A9280035010008ED
:04A92C00110100080D
:10A9300002040608000000000102030401020304EF
:10A94000060708090100000000A24A041A03530088
:10A9500054004D00330032000000000000000000F1
:10A960000000000000000000B1830008317E0008F4
:10A97000317E0008317E0008317E0008317E0008FB
:10A98000317E0008317E0008317E00088D8300088A
:10A99000317E0008317E0008317E0008317E0008DB
:10A9A00074A6000843000000B7A6000812000000CB
:10A9B000E585000809860008098500081D8500084E
:10A9C0002185000889850008B9850008E986000806
:10A9D000F586000801870008000000004000000024
:10A9E00004010000C9A6000804000000E9A6000850
:10A9F00016000000CDA600081C0000001C0000206E
:10AA00001A000000317E0008E5840008317E00084D
:10AA1000317E0008317E0008317E0008317E00085A
:10AA2000317E0008FD84000800C20100000008001B
:10AA300001000000080100200000000000000000EC
:10AA40000000000000000000000000000000000006
:10AA500000000000000000000000000000000000F6
:10AA600000000000000000000000000000000000E6
:10AA700000000000000000000000000000000000D6
:10AA800000000000000000000000000000000000C6
:10AA900000000000000000000000000000000000B6
:10AAA00000000000000000000000000000000000A6
:10AAB0000000000000000000000000000000000096
:10AAC0000000000000000000000000000000000086
:10AAD0000000000000000000000000000000000076
:10AAE0000000000000000000000000000000000066
:10AAF0000000000000000000000000000000000056
:10AB00000000000000000000000000000000000045
:10AB10000000000000000000000000000000000035
:08AB200000000000000000002D
:0400000508005F4947
:00000001FF
